:100000000C9408060C9430060C9430060C943006C0
:100010000C9430060C9430060C9430060C94300688
:100020000C9430060C9430060C9430060C94300678
:100030000C9430060C9430060C9430060C94300668
:100040000C9430060C9430060C94794A0C943006CB
:100050000C94864C0C94CD4C0C9430060C943006C9
:100060000C9430060C9430060C945A450C943006CF
:10007000485454502F312E3020323030204F4B0D09
:100080000A436F6E74656E742D547970653A2074EE
:100090006578742F68746D6C0D0A507261676D61BC
:1000A0003A206E6F2D63616368650D0A0D0A003C8E
:1000B0006D657461206E616D653D76696577706F01
:1000C000727420636F6E74656E743D227769647418
:1000D000683D363430223E0D0A00485454502F31CA
:1000E0002E302034303120556E617574686F72691E
:1000F0007A65640D0A436F6E74656E742D54797061
:10010000653A20746578742F68746D6C0D0A0D0A59
:100110003C68313E34303120556E617574686F72C1
:10012000697A65643C2F68313E0077696E646F7749
:100130002E6C6F636174696F6E3D222F223B3C2FE2
:100140007363726970743E0A006376007670006DA6
:100150007000647000637000677000766F00636FFA
:1001600000736E0070730076730063730076720024
:10017000637200706E00244600244400244400246E
:10018000460024463C6D65746120687474702D656A
:10019000717569763D2272656672657368222063A7
:1001A0006F6E74656E743D22313B2075726C3D2F0D
:1001B000223E0024463C7363726970743E616C6534
:1001C000727428224F7074696F6E732076616C753B
:1001D00065732073617665642E22293B24460024D2
:1001E000463C7363726970743E616C657274282258
:1001F0004E65772070617373776F726473206D75CD
:100200007374206D617463682122293B77696E6481
:100210006F772E6C6F636174696F6E3D222F766FFE
:10022000223B3C2F7363726970743E0A0024463C83
:100230007363726970743E616C65727428224E65D6
:10024000772070617373776F7264207365742E22E8
:10025000293B24460024463C7363726970743E61F6
:100260006C657274282256616C756573206F7574A5
:10027000206F6620626F756E642122293B77696E5C
:10028000646F772E6C6F636174696F6E3D222F7699
:100290006F223B3C2F7363726970743E0A002446E0
:1002A0003C7363726970743E2446005265626F6FDE
:1002B00074696E672E2E2E0024463C6D6574612095
:1002C000687474702D65717569763D227265667209
:1002D0006573682220636F6E74656E743D222444DA
:1002E0003B2075726C3D2F223E003C736372697037
:1002F00074207372633D22766965776F702E6A731E
:10030000223E3C2F7363726970743E0A003C2F7367
:1003100063726970743E0A00305D3B766172206ED4
:100320006F7074733D24442C6C6F633D2224532200
:100330003B00222446222C24442C24442C24442CEC
:10034000003C7363726970743E766172206F7074E2
:10035000733D5B0024462446003C736372697074ED
:10036000207372633D22686F6D652E6A73223E3C76
:100370002F7363726970743E0A003C736372697014
:1003800074207372633D22706E2E6A73223E3C2F7E
:100390007363726970743E0A000A766172206C722F
:1003A000756E3D5B24442C24442C24442C244C5D49
:1003B0003C2F7363726970743E0A005B302C305DB1
:1003C0005D3B0A76617220656E3D24442C72643D6B
:1003D00024442C72733D24442C6D6D3D24442C72B6
:1003E0006473743D244C2C6D61733D24442C7572F0
:1003F000733D24442C776C3D24442C697061733D1B
:1004000024442C6C6F633D222453223B005B244424
:100410002C244C5D2C00305D3B7661722070733D66
:100420005B0024442C00766172206E6272643D246D
:10043000442C747A3D24442C73626974733D5B00D0
:100440003C7363726970743E766172207665723DAA
:1004500024442C646576743D244C3B0A00244624D5
:10046000460077696E646F772E6C6F636174696F95
:100470006E3D222F7670223B3C2F7363726970743D
:100480003E0A00616C657274282250726F67726157
:100490006D202444206D6F64696669656422293B80
:1004A00000616C65727428224E65772070726F67E8
:1004B00072616D2061646465642E22293B002446CC
:1004C0003C7363726970743E003C7363726970744C
:1004D000207372633D22706C6F7470726F672E6A46
:1004E00073223E3C2F7363726970743E0A003C7342
:1004F0006372697074207372633D22706E2E6A732A
:10050000223E3C2F7363726970743E0A00305D3B7B
:100510000024442C00766172206D61736F703D5B26
:100520000024463C7363726970743E766172207376
:1005300065713D24442C6D61733D24442C776C3DE2
:1005400024442C7364743D24442C6D746F6E3D24DC
:10055000442C6D746F66663D24442C64657664613A
:10056000793D24442C6465766D696E3D24442C6489
:10057000643D24442C6D6D3D24442C79793D244404
:100580003B0024463C7363726970743E77696E6405
:100590006F772E6C6F636174696F6E3D222F76707A
:1005A000223B3C2F7363726970743E0A003C736394
:1005B00072697074207372633D226D6F6470726F24
:1005C000672E6A73223E3C2F7363726970743E0A11
:1005D000003C2F7363726970743E0A3C73637269E6
:1005E0007074207372633D22706E2E6A73223E3CDB
:1005F0002F7363726970743E0A005D3B002C2444C3
:10060000007661722070726F673D5B24442C244435
:100610002C24442C24442C24442C24442C244400F6
:100620003C7363726970743E766172206E626F61B2
:100630007264733D24442C7069643D24442C6970B9
:1006400061733D24443B0024462446003C7363729E
:10065000697074207372633D227669657770726F7A
:10066000672E6A73223E3C2F7363726970743E0A70
:10067000003C736372697074207372633D22706E04
:100680002E6A73223E3C2F7363726970743E0A00B7
:10069000244624463C7363726970743E0024463CD1
:1006A0007363726970743E2446003C7363726970B0
:1006B00074207372633D2276696577726F2E6A7358
:1006C000223E3C2F7363726970743E0A003C736370
:1006D00072697074207372633D22706E2E6A732289
:1006E0003E3C2F7363726970743E0A00305D3B3C80
:1006F0002F7363726970743E0A0024442C002446F0
:1007000024463C7363726970743E766172206E6237
:100710006F617264733D24442C6D61733D24442CDD
:10072000697061733D24442C6475723D5B003C73B9
:100730006372697074207372633D707324442E6A0F
:10074000733E3C2F7363726970743E0A003C2F73D2
:1007500063726970743E0A00766172206E70726F07
:1007600067733D24442C6E626F617264733D244450
:100770002C697061733D24442C6D6E703D24442CB3
:1007800070643D5B5D3B002446005D3B002C2444CF
:100790000070645B24445D3D5B24442C24442C2481
:1007A000442C24442C24442C24442C24440024464B
:1007B0003C7363726970743E616C65727428224385
:1007C00068616E6765732073617665642E22293BCC
:1007D00024460024467661722000305D3B3C2F7336
:1007E00063726970743E0A3C73637269707420733B
:1007F00072633D2276696577736E2E6A73223E3C82
:100800002F7363726970743E0A0024442C00766171
:1008100072206D61736F703D5B0024463C736372A0
:100820006970743E766172206E626F617264733DAE
:1008300024442C6D61786C656E3D24442C6D61738D
:100840003D24442C697061733D24442C0027275DAE
:100850003B0A00272453272C00736E616D65733D9E
:100860005B00436F6E6E656374696E672E2E2E009B
:10087000446574656374696E67207553442E2E2E2B
:10088000000001080006040001450000820000404D
:10089000002000504F535420244620485454502FD9
:1008A000312E300D0A486F73743A2024460D0A2405
:1008B0004624534163636570743A202A2F2A0D0A37
:1008C000436F6E74656E742D4C656E6774683A2064
:1008D00024440D0A436F6E74656E742D54797065EF
:1008E0003A206170706C69636174696F6E2F782D46
:1008F0007777772D666F726D2D75726C656E636F8D
:100900006465640D0A0D0A245300474554202446AB
:10091000245320485454502F312E300D0A486F7301
:10092000743A2024460D0A24460D0A0D0A0041633C
:10093000636570743A20746578742F68746D6C0008
:10094000E30004FA0001000000014669726D77615E
:100950007265207665722E0054696D65207A6F6E1F
:10096000653A004E54502053796E633A00557365D2
:1009700020444843503A005374617469632E69708F
:10098000313A006970323A006970333A0069703464
:100990003A00476174657761792E6970313A006970
:1009A00070323A006970333A006970343A00485442
:1009B000545020706F72743A00004175746F207249
:1009C00065636F6E6E6563743A004578702E2062C1
:1009D0006F617264733A0053657175656E74696115
:1009E0006C3A0053746174696F6E2064656C617950
:1009F0003A004D61737465722073746174696F6E2F
:100A00003A004D61732E206F6E2061646A2E3A00A9
:100A10004D61732E206F66662061646A2E3A005520
:100A20007365207261696E2073656E736F723A0030
:100A30004E6F726D616C6C79206F70656E3A002537
:100A40002057617465722074696D653A0053656C56
:100A500066746573742074696D653A0049676E6FDA
:100A600072652070617373776F72643A00446576C3
:100A70006963652049443A004C434420436F6E74D7
:100A8000726173743A004C4344204261636B6C6939
:100A90006768743A004E5450207365727665722E02
:100AA0006970313A006970323A006970333A00690E
:100AB00070343A00526573657420616C6C3F004D70
:100AC0006F6E005475650057656400546875004684
:100AD0007269005361740053756E00206D696E0079
:100AE000207365630025004E6F00596573002B006D
:100AF0002B0020474D54003030003A002D002B00D1
:100B00000020202020002D5261696E2053746F70E8
:100B10002D002D44697361626C6564212D003A00DB
:100B200045004D433A003A002E002D0020002020C1
:100B3000003A00200042333A686F6C6420746F20E2
:100B4000736176650042333A73656C2042312F42FF
:100B5000323A636867003D3D536574204F70746995
:100B60006F6E733D3D00506C656173652057616920
:100B7000742E2E2E00526573657474696E6720455D
:100B80004550524F4D0000002100240027002A004C
:100B900000002200250028002B0000002000230078
:100BA00026002900020202020202020204040404D6
:100BB0000404040403030303030303030101010109
:100BC0000101010101020408102040800102040813
:100BD0001020408001020408102040808040201036
:100BE00008040201000000010200000000000000F3
:100BF00004030706000000000000000000000000E1
:100C0000000000001A089220083B903CF643AD4DCE
:100C100011241FBECFEFD0E1DEBFCDBF12E0A0E0B8
:100C2000B1E0E2E4FFE902C005900D92A03DB107FA
:100C3000D9F71DE0A0EDB2E001C01D92A531B107CA
:100C4000E1F71CE0C0E1DCE004C02297FE010E9455
:100C5000644FC430D107C9F70E94794B0C949F4F61
:100C60000C940000FC0188279927E89421912032F8
:100C7000E9F3293010F02E30C8F32B3241F02D3239
:100C800039F4689404C00E94E406820F911D2191FA
:100C900020532A30C0F31EF4909581959F4F0895FC
:100CA000FB01DC0102C005900D9241505040D8F785
:100CB0000895FB01DC0104C08D910190801921F49D
:100CC00041505040C8F7881B990B0895DC0101C0C2
:100CD0006D9341505040E0F70895FB01DC018D9188
:100CE000019080190110D9F3990B0895FB01DC01E3
:100CF00001900D920020E1F70895FB01DC014150C5
:100D0000504030F08D910190801919F40020B9F70E
:100D1000881B990B0895A0E0B0E0E1E9F6E00C949F
:100D2000724F7C01EB018A01690109C0CE01219655
:100D3000F6010995F70181937F01015010400115DB
:100D40001105A1F7CDB7DEB7E8E00C948E4FA0E017
:100D5000B0E0EDEAF6E00C94724FEC017B018A0101
:100D6000690109C0CE012196F70161917F01F60169
:100D700009950150104001151105A1F7CDB7DEB757
:100D8000E8E00C948E4FFB019F01E8944230C4F0E0
:100D90004532B4F44A3029F497FB1EF490958195BE
:100DA0009F4F642F77270E94194F805D8A330CF084
:100DB000895D8193CB010097A1F716F45DE2519311
:100DC0001082C9010C9411077AE0979F902D879F9C
:100DD000802D910D11240895FA01CF93FF93EF9385
:100DE0002230CCF02532BCF4C22F2C2F33274427DD
:100DF0005527FF93EF930E94404FEF91FF91605D65
:100E00006A330CF0695D6193B901CA0160507040AA
:100E10008040904051F710828F919F91CF910C9418
:100E20001107DC01FC01672F71917723E1F73297FD
:100E300004C07C916D9370836291AE17BF07C8F3B5
:100E400008959C01F999FECF32BD21BDF89A80B575
:100E500008959C01F999FECF1FBA32BD21BD60BD36
:100E60000FB6F894FA9AF99A0FBE0895FC01A6817C
:100E7000B7816D93B783A68381E090E00895CF9208
:100E8000DF92EF92FF920F931F93CF93DF937B013B
:100E90008C010894E11CF11C011D111DC090910BE7
:100EA000442361F430918E0B36953695369531702A
:100EB000ACE5B7E0CCE9D6E0DD2475C020918E0B1F
:100EC0002695269526952170ECE5F7E0CCE9D6E04D
:100ED0006C2D70E0660F771F660F771F6E0F7F1FF8
:100EE0008CE3D82E27C080819181A281B3810097A5
:100EF000A105B105E9F0E882F9820A831B83A80104
:100F00009701280F391F4A1F5B1F208331834283BB
:100F10005383809104028D9DC00111247C01002720
:100F2000F7FC0095102FE20EF31E041F151F21E0A1
:100F300034962496E617F707B1F62170220F220F98
:100F4000220F80918E0B877F822B37C04D915D9150
:100F50006D917C911397411551056105710501F162
:100F6000ED2DE695E695E695F0E0EE56F44F80819E
:100F700090E02D2D277002C0959587952A95E2F770
:100F800080FD0EC0E882F9820A831B834E0D5F1D2F
:100F9000601F711F4D935D936D937C93139731E0A8
:100FA000D39414962496DC1488F23170330F330FE7
:100FB000330F80918E0B877F832B80938E0BDF9175
:100FC000CF911F910F91FF90EF90DF90CF900895F8
:100FD000ACE1B8E080E090E0FC01E456F94F10820B
:100FE000118212821382FC01E45AF84F108211829E
:100FF000128213821D920496803C910569F7F9993B
:10100000FECF86ED93E092BD81BDF89A80B58093C6
:1010100093061092940610929506109297061092DD
:101020009606109298061092990610929A061092BF
:101030009B06089510928A06109289068BE692E02C
:10104000909388068093870608959F92AF92BF92EF
:10105000CF92DF92EF92FF920F931F93CF93DF9384
:10106000EC01962E8AE598E0BE010E94E5238823D4
:1010700009F456C08AE598E0BE0141E00E94CB2405
:10108000AA24BB2465018AE598E00E94C620EC01F1
:10109000ABE9B8E026E330E040E050E0A20EB31E3A
:1010A000C41ED51EF501EE52FD4F2AEC3FEF4FEF67
:1010B0005FEFA20EB31EC41ED51E8601750107C0C8
:1010C0000894E11CF11C011D111D8D918193C70134
:1010D0008A199B098C179D079CF330E0E31632E0D8
:1010E000F30630E0030730E0130740F0C70160E18A
:1010F0000E940F2FAA24BB24650109C041E0941669
:1011000021F4C70161E10E940F2F57016801C0500F
:10111000D24009F4B8CF8AE598E00E948B2081E0A4
:10112000DF91CF911F910F91FF90EF90DF90CF90C3
:10113000BF90AF909F900895BF92CF92DF92EF92B1
:10114000FF920F931F93CF93DF932DB73EB72E508F
:1011500030400FB6F8943EBF0FBE2DBFEDB7FEB7BF
:10116000319607E816E0ADB7BEB712961C930E9302
:1011700011978EEF96E09383828380E790E09583CA
:1011800084838FEA90E0978386838091900B808799
:101190001186809109028287138680912C028487B0
:1011A00015860E94DA2CDD2420E7E22E23E0F22EC1
:1011B000EDB7FEB73E960FB6F894FEBF0FBEEDBF7B
:1011C000B02EC12E0AEF16E033C0F999FECFF2BC63
:1011D000E1BCF89A90B5F999FECF0894E11CF11C96
:1011E000F2BCE1BCF89A80B5D92FC0E000D000D0A5
:1011F00000D0EDB7FEB73196ADB7BEB71196BC9231
:1012000011971296CC92138302839E01280F311DF1
:10121000358324830E94DA2CD3940894E11CF11CBA
:101220008DB79EB706960FB6F8949EBF0FBE8DBFC2
:101230008091910BD81608F4C8CF00D000D007E8F1
:1012400016E0ADB7BEB712961C930E9311978CEEB5
:1012500096E014969C938E9313970E94DA2CEDB728
:10126000FEB7128301838DEC96E0948383830E9402
:10127000DA2CADB7BEB712961C930E9311978AEA7B
:1012800096E014969C938E9313970E94DA2C0F90FD
:101290000F900F900F9081E0DF91CF911F910F91F0
:1012A000FF90EF90DF90CF90BF900895CF92DF92A4
:1012B000EF92FF920F931F93DF93CF9300D000D054
:1012C000CDB7DEB70E94CD4A7B018C016E01089438
:1012D000C11CD11C0E943C380E944731C60160915C
:1012E0004D010E94352E8823E1F0E980FA800B81C0
:1012F0001C8180EC98EDA4E5BCE7E80EF91E0A1FFE
:101300001B1F6091B40170E080E090E024E833E0BE
:1013100040E050E00E94EE4EE60EF71E081F191F37
:101320000EC00E94CD4A6E197F09800B910B685E3A
:1013300073408040904070F2EE24FF248701B70193
:10134000C8010F900F900F900F90CF91DF911F91D8
:101350000F91FF90EF90DF90CF900895EF92FF9262
:101360001F93DF93CF9300D000D0CDB7DEB780912D
:1013700040028983809145028A8380914A028B834F
:1013800080914F028C8310E07E010894E11CF11CD7
:1013900060914D016F5F60934D01C7010E94A930BC
:1013A0006AEF70E080E090E00E94DB4A0E945609FC
:1013B0009B01AC01611571058105910519F41F5F51
:1013C0001A3031F7B901CA010F900F900F900F90AA
:1013D000CF91DF911F91FF90EF900895CF93DF930E
:1013E0009C0110925606FC01A081B181C0E0D0E0C2
:1013F0000FC09C919D3231F09B3221F0892F805398
:101400008A3068F4FE01EA5AF94F908321961196CA
:10141000F901808191810A96A817B90750F3CA5A39
:10142000D94F18821196F901B183A08386E596E021
:101430000E943206DF91CF910895AF92BF92CF9272
:10144000DF92EF92FF920F931F93CF93DF938DB7AD
:101450009EB708970FB6F8949EBF0FBE8DBFEDB72D
:10146000FEB7319607E816E0ADB7BEB712961C93EB
:101470000E93119784E593E09383828380E790E055
:10148000958384838FEA90E0978386830E94DA2C89
:101490000F900F900F900F90EDB7FEB7128301835E
:1014A00081E493E0948383830E94DA2C4FEAE42E54
:1014B00041E0F42EDD24C0E0D0E00F900F900F90BB
:1014C0000F90B02EC12E02E313E07C2FAD2ED7017A
:1014D00014968C91149781FF3CC012964D915C91AB
:1014E000139711966C9111978C91C43129F4282F80
:1014F00030E02C53304002C0282F30E0EDB7FEB76B
:101500003C970FB6F894FEBF0FBEEDBF3196ADB756
:10151000BEB71196BC9211971296CC921383028398
:101520005583448380E090E0613011F481E090E0E5
:1015300097838683318720877287A3860E94DA2C5F
:10154000D394EDB7FEB73C960FB6F894FEBF0FBE2E
:10155000EDBF219685E090E0E80EF91EC232D1057C
:1015600009F0B3CF36E5E32E36E0F32E80E590E0C8
:10157000B7010E945E3CADB7BEB718970FB6F8949E
:10158000BEBF0FBEADBFEDB7FEB7319607E816E0A0
:1015900012961C930E93119788E193E093838283B4
:1015A000D4821582F782E6820E94DA2C0F900F9087
:1015B0000F900F90EDB7FEB7128301838DE093E09B
:1015C000948383830E94DA2CADB7BEB712961C9326
:1015D0000E9311978AEE92E014969C938E93139734
:1015E0000E94DA2C0F900F900F900F9081E0DF9106
:1015F000CF911F910F91FF90EF90DF90CF90BF9010
:10160000AF9008954F925F926F927F928F929F92C8
:10161000AF92BF92CF92DF92EF92FF920F931F9300
:10162000DF93CF930F92CDB7DEB70E94D5365B0123
:101630006C012DB73EB7285030400FB6F8943EBF2E
:101640000FBE2DBFEDB7FEB7319607E816E0ADB778
:10165000BEB712961C930E9311978DE594E0938379
:10166000828380E790E0958384838FEA90E097837C
:1016700086830E94DA2C00D0EDB7FEB73196ADB765
:10168000BEB712961C930E93119780E494E0938357
:10169000828389EC90E095838483A682B782C0869A
:1016A000D1860E94DA2C0F900F90EDB7FEB73196DD
:1016B000ADB7BEB712961C930E93119786E294E0D5
:1016C000938382838091900B848315828091B401EF
:1016D000868317820E94DA2C90E0EDB7FEB7389629
:1016E0000FB6F894FEBF0FBEEDBF780102E214E022
:1016F00023C000D000D000D0EDB7FEB73196ADB713
:10170000BEB71196EC9211971296FC921383028346
:10171000A92FB0E0AE56B44F8C9184831582998383
:101720000E94DA2C99819F5FEDB7FEB736960FB60F
:10173000F894FEBF0FBEEDBF8091900BA7E86A2E14
:10174000A6E07A2E9817A8F200D000D0ADB7BEB7A9
:1017500012967C926E92119786E194E014969C9377
:101760008E9313970E94DA2C99240F900F900F906C
:101770000F90C301762C892EFDE04F2EF4E05F2EF2
:1017800066C0A92DB0E0FD01E45EF74F60816623DD
:10179000A9F1CD01880F991F880F991FFC01E4560C
:1017A000F94FE080F18002811381FC01E45AF84F87
:1017B000AE14BF04C006D10648F0208131814281B9
:1017C00053812A193B094C095D0908C020813181E8
:1017D000428153812E193F09400B510BAA0FBB1FA9
:1017E000AA0FBB1FA45AB84F8D919D910D90BC912B
:1017F000A02D8E5F9F4FAF4FBF4F21F420E030E010
:1018000040E050E08DB79EB70A970FB6F8949EBFA0
:101810000FBE8DBFEDB7FEB73196ADB7BEB711960F
:101820007C92119712968C92538242826483158225
:1018300026833783408751870E94DA2C9394EDB733
:10184000FEB73A960FB6F894FEBF0FBEEDBF80917B
:10185000910B981608F495CF56E5E52E56E0F52E37
:1018600080E590E0B7010E945E3C2DB73EB72A515B
:1018700030400FB6F8943EBF0FBE2DBFEDB7FEB798
:10188000319607E816E0ADB7BEB712961C930E93DB
:1018900011978BEB93E09383828380918E0B817001
:1018A0008483158280918E0B869581708683178242
:1018B00080918E0B869586958170808711868091A8
:1018C0008E0B829581708287138680919E0B9091FA
:1018D0009F0BA091A00BB091A10B84879587A68741
:1018E000B78780910902808B118A80911802828BC0
:1018F000138A80912202848B158A80912C02868B18
:10190000178AF18EE08E0E94DA2CEDB7FEB73C9676
:101910000FB6F894FEBF0FBEEDBF3196ADB7BEB7A0
:1019200012961C930E93119789E993E09383828317
:101930008091940684831582809195068683178210
:10194000809196069091970691878087809198065E
:1019500090919906A0919A06B0919B0682879387F1
:10196000A487B5870E94DA2CEDB7FEB73A960FB67A
:10197000F894FEBF0FBEEDBF128301838AE793E0A8
:10198000948383830E94DA2CADB7BEB712961C9362
:101990000E93119789E593E014969C938E93139779
:1019A0000E94DA2C81E00F900F900F900F900F9013
:1019B000CF91DF911F910F91FF90EF90DF90CF902B
:1019C000BF90AF909F908F907F906F905F904F905F
:1019D0000895FF920F931F93CF93DF938C01AC0177
:1019E0004B5F5F4FDC0115968C91803221F4CA0168
:1019F0000E94020B6CC0CEE4D1E0A0E0B0E0682F02
:101A0000772767FD7095FA2EE881F981849190E03F
:101A10008617970709F068C03196249130E0FA01E3
:101A20008181992787FD90952817390709F05CC0B7
:101A3000AA0FBB1FAA0FBB1FA05BBE4FED91FC916D
:101A4000CA010995882301F500D000D000D0EDB778
:101A5000FEB7319687E896E0ADB7BEB712969C9375
:101A60008E93119786E791E0938382838AED90E0CD
:101A7000958384830E94DA2CEDB7FEB736960FB6B5
:101A8000F894FEBF0FBEEDBFFFE0FF1601F5402F3B
:101A9000E6E5F6E0C801DC0101C081939A2F941BB2
:101AA00015968C911597803229F0119626E0E6372D
:101AB000F20799F7E92FF0E0EA5AF94F10820E94F5
:101AC000922F86E596E061E00E94250815C080917E
:101AD0008D0690918E0620918B0630918C06821B8C
:101AE000930B0E94C52F08C0F39411962496AF3033
:101AF000B10509F088CFC8CFDF91CF911F910F9129
:101B0000FF900895BF92CF92DF92EF92FF920F93D2
:101B10001F936C01FC01B080E1800E94D53620E863
:101B200031E541E050E00E94404F8B2D8F77280F28
:101B3000311D411D511DFF2400E010E0CA01B90113
:101B4000A80197010E94404FF0E8BF22B62AF60193
:101B5000B0821F910F91FF90EF90DF90CF90BF90D8
:101B600008956F927F928F929F92AF92BF92CF9281
:101B7000DF92EF92FF920F931F934C01FC01708054
:101B800061800E94D536A62CBB24CC24DD242FE70F
:101B9000E22EE720FF24E60CF11C0027F7FC00955D
:101BA000102F20E831E541E050E00E94404FCA018B
:101BB000B901A60195010E94404FE61AF70A080BE9
:101BC000190BC801B701A60195010E94404FF0E82A
:101BD0007F22762AF40170821F910F91FF90EF907F
:101BE000DF90CF90BF90AF909F908F907F906F903D
:101BF0000895EF92FF921F93CF93DF93182F7B01ED
:101C00000E94D5369B01AC01C12FD0E02F5F3F4F22
:101C10004F4F5F4FCE01880F991F880F991FFC010E
:101C2000E456F94F2083318342835383FC01E45A05
:101C3000F84FE114F10449F48EEF9FEFAFEFBFEFDF
:101C400080839183A283B3830DC0C701AA2797FD28
:101C5000A095BA2F280F391F4A1F5B1F208331839D
:101C600042835383C45ED74F83E6888380918E0B73
:101C7000886080938E0BDF91CF911F91FF90EF9042
:101C800008958F929F92AF92BF92CF92DF92EF9280
:101C9000FF920F931F93CF93DF938C010E5F1F4F23
:101CA00020E030E006C0F901EB5AF94F90830F5F56
:101CB0001F4FE22FD8019C91892F80538A3028F43E
:101CC0002F5F3F4F2530310571F7F0E0EA5AF94FA9
:101CD000108286E596E00E943206EC0197FD00C175
:101CE0008091910B90E08C179D070CF4F9C0F801DE
:101CF00080818D3309F057C0209709F4F1C080919D
:101D00008E0B84FFEDC02197C801019621812033FD
:101D100079F40E94D536EC2FF0E0EE0FFF1FEE0FA6
:101D2000FF1FE45AF84F608371838283938319C045
:101D3000213309F0D5C066E576E040E320E031E0EC
:101D40000E94D633882319F460E070E007C086E56E
:101D500096E00E943206BC0197FDC2C08C2F0E9403
:101D6000F90D00D000D000D0EDB7FEB7319687E86E
:101D700096E0ADB7BEB712969C938E93119782E80A
:101D800091E09383828380E790E0958384830E942F
:101D9000DA2C81E0EDB7FEB736960FB6F894FEBFA9
:101DA0000FBEEDBF9EC000D000D000D0EDB7FEB793
:101DB000319687E896E0ADB7BEB712969C938E93A6
:101DC00011978FE791E09383828380E790E095837A
:101DD00084830E94DA2CEDB7FEB736960FB6F894DE
:101DE000FEBF0FBEEDBF209721F48091910B90E0D4
:101DF00003C08C2F9C2F9150C0E0D0E0E92EFF242F
:101E0000082F10E037E8C32E36E0D32E29E7822EC4
:101E100021E0922E9CE7A92E91E0B92E58C0909116
:101E20008E0B90FF39C091FD37C080911802882336
:101E300011F092FD31C000D000D000D0ADB7BEB7D8
:101E40001196EDB7FEB7D282C1821396BC92AE92C4
:101E50001297F90183E0F595E7958A95E1F7EE563B
:101E6000F44F808190E02770307002C0959587957F
:101E70002A95E2F78170907015969C938E93149733
:101E80000E94DA2C2DB73EB72A5F3F4F0FB6F89469
:101E90003EBF0FBE2DBF1AC000D000D000D0EDB79E
:101EA000FEB73196ADB7BEB71296DC92CE921197BF
:101EB00093828282158214820E94DA2CEDB7FEB7DB
:101EC00036960FB6F894FEBF0FBEEDBF21969E0169
:101ED0002E0D3F1D201731070CF4A1CF81E001C06A
:101EE00080E0DF91CF911F910F91FF90EF90DF90F5
:101EF000CF90BF90AF909F908F900895DF92EF9218
:101F0000FF920F931F93CF93DF9300D000D007E889
:101F100016E0ADB7BEB712961C930E93119789E5E4
:101F200098E014969C938E9313970E94DA2CFF24CA
:101F30000F900F900F900F90D02EE12E06E516E037
:101F4000C3E5D8E021C08F2D66E576E00E945F3BB7
:101F500000D000D000D0EDB7FEB73196ADB7BEB718
:101F60001196DC9211971296EC92D383C28315835B
:101F700004830E94DA2CF394EDB7FEB736960FB6C1
:101F8000F894FEBF0FBEEDBF8091910BF816D8F20A
:101F900000D000D087E896E0ADB7BEB712969C930C
:101FA0008E9311978DE498E014969C938E931397DB
:101FB0000E94DA2C0F900F900F900F90DF91CF912D
:101FC0001F910F91FF90EF90DF90089500D000D007
:101FD00000D0EDB7FEB7319687E896E0ADB7BEB753
:101FE00012969C938E93119783ED97E0938382834F
:101FF00080E790E0958384830E94DA2C8DB79EB7AA
:1020000006960FB6F8949EBF0FBE8DBF0E947E0F3E
:1020100081E00895CF92DF92FF920F931F93DF9399
:10202000CF930F92CDB7DEB72DB73EB72E503040CD
:102030000FB6F8943EBF0FBE2DBFEDB7FEB7319679
:1020400007E816E0ADB7BEB712961C930E93119732
:102050008AE198E09383828380E790E0958384838C
:102060008091900B8683178280E190E09187808732
:10207000809109028287138680912C0284871586BD
:102080000E94DA2CEDB7FEB73E960FB6F894FEBF6D
:102090000FBEEDBF0E947E0F00D000D0ADB7BEB71F
:1020A00012961C930E9311978EE098E014969C93D1
:1020B0008E9313970E94DA2C90E00F900F900F9060
:1020C0000F90F02E012F5AE0C52E58E0D52E23C0D8
:1020D00000D000D000D0EDB7FEB73196ADB7BEB797
:1020E0001196FC92119712960C93D382C282A92F5B
:1020F000B0E0A856B44F8C918483158299830E94D6
:10210000DA2C99819F5FEDB7FEB736960FB6F8943B
:10211000FEBF0FBEEDBF8091900B9817C8F200D0A4
:1021200000D087E896E0ADB7BEB712969C938E9329
:1021300011978AED97E014969C938E9313970E94C3
:10214000DA2C81E00F900F900F900F900F90CF91AD
:10215000DF911F910F91FF90DF90CF9008959C0128
:1021600080912C02882311F081E00895C90166E571
:1021700076E040E322E031E00E94D633882331F05C
:1021800086E596E00E94713C811181E008956F928E
:102190007F928F929F92AF92BF92CF92DF92EF92F7
:1021A000FF920F931F93DF93CF93CDB7DEB7E597E1
:1021B0000FB6F894DEBF0FBECDBF73E0A72EB12CD3
:1021C000A80EB91EC5010E94AF10882309F402C1F0
:1021D0000FEA11E0EE24CC24DD244E010894811C8A
:1021E000911C62E0662E712C6C0E7D1E2C2D9D2D97
:1021F000D80114968C91149781FF3BC011968C9155
:102200001197813009F41C92D401EFE6F2E085E0E9
:1022100001900D928150E1F7822FB3014AE050E026
:102220000E94C306C50166E576E040E394010E9482
:10223000D6338823F1F0F801F180F1E0FF1619F4AC
:10224000D801FC9216C086E596E00E9432069C01F9
:10225000B4E1CB1611F4245C3F4F37FD08C08F2D3D
:1022600090E0821793071CF0F801208302C0EE244F
:10227000E3940894C11CD11C0B5F1F4FF2E2CF16F0
:10228000D10409F0B3CFC50166E576E040E325E06F
:1022900031E00E94D633882351F086E596E00E9413
:1022A000223480E590E066E576E00E94393CEE203D
:1022B00089F000D000D000D0EDB7FEB7319687E8A6
:1022C00096E0ADB7BEB712969C938E93119785E5B5
:1022D00092E0A5C00E94153CC50166E576E040E3AA
:1022E00029E031E00E94D633882309F440C08E01F2
:1022F0000A5F1F4FC501B80140E32DE031E00E94A5
:10230000D633882309F47BC086E596E0B80140E126
:1023100050E00E947D06009709F071C080E490E0D3
:1023200066E576E00E94393C2DB73EB72850304034
:102330000FB6F8943EBF0FBE2DBFEDB7FEB7319676
:1023400087E896E0ADB7BEB712969C938E9311972F
:102350008DE292E09383828380E790E0958384838B
:102360008AE291E0978386830E94DA2C2AC02DB7F7
:102370003EB7285030400FB6F8943EBF0FBE2DBF79
:10238000EDB7FEB7319687E896E0ADB7BEB71296C7
:102390009C938E93119783EB91E09383828380E7E4
:1023A00090E0958384838AE291E0978386830E94FC
:1023B000DA2C10928F0610929006109291061092CD
:1023C000920681E0EDB7FEB738960FB6F894FEBFDF
:1023D0000FBEEDBFE5960FB6F894DEBF0FBECDBFC2
:1023E000CF91DF911F910F91FF90EF90DF90CF90F1
:1023F000BF90AF909F908F907F906F90089500D086
:1024000000D000D0EDB7FEB7319687E896E0ADB7C3
:10241000BEB712969C938E9311978FED91E09383A4
:10242000828380E790E0958384830E94DA2C81E0A8
:10243000EDB7FEB73696C9CF8F929F92AF92BF92FB
:10244000CF92DF92FF920F931F93DF93CF9300D031
:1024500000D0CDB7DEB7A3E0CA2ED12CC80ED91E4E
:10246000C6010E94AF10882309F483C083E78983E3
:102470001A821B821C8210E0F2E08F2E912C8C0EAF
:102480009D1E5E010894A11CB11C1AC0812F90E012
:10249000B4014AE050E00E94C306C60166E576E05A
:1024A00040E395010E94D633882349F086E596E003
:1024B0000E942234812F66E576E00E94843B1F5FF4
:1024C0008091910B181710F38DE68983FF24E2E0C9
:1024D0008E2E912C8C0E9D1E5E010894A11CB11CA9
:1024E0001AC00F2D10E0C801B4014AE050E00E946C
:1024F000C306C60166E576E040E395010E94D63347
:10250000882341F086E596E00E9432060856144F73
:10251000D8018C93F3948091900BF81610F30E94DD
:10252000AE3BEDB7FEB738970FB6F894FEBF0FBEBF
:10253000EDBF319687E896E0ADB7BEB712969C9393
:102540008E9311978EEA97E09383828380E790E0E1
:10255000958384838AE291E0978386830E94DA2CB4
:1025600081E0EDB7FEB738960FB6F894FEBF0FBE08
:10257000EDBF0F900F900F900F90CF91DF911F91B3
:102580000F91FF90DF90CF90BF90AF909F908F9072
:1025900008958F929F92AF92BF92CF92DF92EF9267
:1025A000FF920F931F93CF93DF93EC017A018B017E
:1025B000CB01BA010E94C2354C01C801B7010E948B
:1025C000BC355C018889882309F481C0D880D7FE96
:1025D00021C0C98021E02C15E8F4C801B70120E82A
:1025E00031E541E050E00E94404FCA01B9012C2D75
:1025F00030E040E050E00E94404F2FE7D2222D2DE6
:1026000030E040E050E0621773078407950709F057
:102610005EC031C0C801B7010E94B035288130E0EA
:1026200090E0059667E070E00E942D4F02C035955E
:1026300027958A95E2F720FF4AC0C801B7010E949A
:10264000B635D82E888187FF16C08981882319F472
:10265000D0FE11C03CC0813071F48FE1D816B9F1C1
:102660002DE1D21609F042C0C801B7010E94AA3577
:102670000297E1F52CC08CE390E0889E9001899E42
:10268000300D989E300D11242A0D3B1D4A815B812F
:1026900024173507E0F08C819D8182179307B8F0ED
:1026A000EE81FF81309799F0241B350B40E0C90182
:1026B000BF010E94194F6E9FC0016F9F900D7E9FBA
:1026C000900D11248217930719F441E001C040E0F6
:1026D000842FDF91CF911F910F91FF90EF90DF90AA
:1026E000CF90BF90AF909F908F900895D0FCC3CFB4
:1026F000EECF982F9B0180919306981768F461E1C3
:10270000969FB001112468527C4FC90141E150E00D
:1027100021E237E00E948B060895CF92DF92EF927C
:10272000FF920F931F93DF93CF93CDB7DEB76297DE
:102730000FB6F894DEBF0FBECDBF8C010D5F1F4FEB
:10274000C8010E942234C80166E576E040E321E139
:1027500031E00E94D633882309F40BC186E596E068
:102760000E9432067C012FEF8F3F92070CF401C1CB
:102770008091930690E0E816F9060CF0FAC08DB748
:102780009EB708970FB6F8949EBF0FBE8DBFEDB7EA
:10279000FEB7319607E816E0ADB7BEB712961C93A8
:1027A0000E93119787E496E09383828380E790E00D
:1027B000958384838FEA90E0978386830E94DA2C46
:1027C00000D0EDB7FEB73196ADB7BEB712961C93E9
:1027D0000E93119780E296E0938382838091900B11
:1027E00084831582F782E68280912C02808711868D
:1027F0000E94DA2CEDB7FEB73A960FB6F894FEBFFA
:102800000FBEEDBFFFEFEF16FFEFFF0609F48FC01D
:102810008E2D7E010894E11CF11CB7010E947913F2
:102820008A81823018F0C7010E94B10D2DB73EB7E2
:10283000225130400FB6F8943EBF0FBE2DBFEDB70A
:10284000FEB7319607E816E0ADB7BEB712961C93F7
:102850000E93119781E096E0938382838989848324
:1028600015828981868317828A81808711868B8170
:102870009C81938782878D819E81958784878F81B4
:1028800098859787868789859A85918B808B0E940A
:10289000DA2C90E0EDB7FEB772960FB6F894FEBF53
:1028A0000FBEEDBF6801BDEFEB2EB5E0FB2E8E0134
:1028B000055F1F4F22C000D000D000D0EDB7FEB79B
:1028C0003196ADB7BEB71196CC9211971296DC92A5
:1028D000F382E282D801A90FB11D8C918483158205
:1028E0009A8B0E94DA2C9A899F5FEDB7FEB73696D5
:1028F0000FB6F894FEBF0FBEEDBF8091900B9817F6
:10290000D0F200D000D087E896E0ADB7BEB71296FF
:102910009C938E9311978AEF95E014969C938E93D7
:1029200013970E94DA2C0F900F900F900F9000D009
:1029300000D007E816E0EDB7FEB71283018381ED02
:1029400095E0948383830E94DA2CADB7BEB71296CC
:102950001C930E9311978DEA95E014969C938E9399
:1029600013970E94DA2C81E00F900F900F900F9038
:1029700001C080E062960FB6F894DEBF0FBECDBFF7
:10298000CF91DF911F910F91FF90EF90DF90CF904B
:1029900008952F923F925F926F927F928F929F92B3
:1029A000AF92BF92CF92DF92EF92FF920F931F935D
:1029B000DF93CF93CDB7DEB761970FB6F894DEBF44
:1029C0000FBECDBFD82EE82EFF2487E090E0E80EA2
:1029D000F91E4E010894811C911C87E8A82E86E000
:1029E000B82E0BE0202E312C2C0E3D1EC5015A2C8A
:1029F000C92E1AE8612E17E0712E73C08D2DB40117
:102A00000E9479138A81823018F0C4010E94B10DAE
:102A1000ADB7BEB754970FB6F894BEBF0FBEADBFEB
:102A2000EDB7FEB731961296BC92AE92119781E93E
:102A300097E0938382831583048389898683178231
:102A40008981808711868A81828713868B819C8108
:102A5000958784878D819E81978786878F819885CA
:102A6000918B808B89859A85938B828B0E94DA2C3F
:102A700010E0ADB7BEB754961CC000D000D000D057
:102A8000EDB7FEB73196ADB7BEB71296BC92AE9217
:102A900011978DE897E093838283D101A10FB11D37
:102AA0008C91848315820E94DA2C1F5FADB7BEB76C
:102AB00016960FB6F894BEBF0FBEADBF8091900BB7
:102AC0001817D8F200D000D0EDB7FEB75182C282FD
:102AD000748263820E94DA2CD3940F900F900F902F
:102AE0000F900D2D10E0E016F1062CF0809193066A
:102AF000D81608F483CF61960FB6F894DEBF0FBEE8
:102B0000CDBFCF91DF911F910F91FF90EF90DF909C
:102B1000CF90BF90AF909F908F907F906F905F907D
:102B20003F902F900895FF920F931F93CF93DF93C1
:102B30008DB79EB70C970FB6F8949EBF0FBE8DBF92
:102B4000EDB7FEB73196C7E8D6E0ADB7BEB712967F
:102B5000DC93CE93119788E597E0938382838091ED
:102B60009306848315828091900B868317828091CF
:102B70002C02808711868EE390E0938782870E94E3
:102B8000DA2CEDB7FEB73C960FB6F894FEBF0FBE39
:102B9000EDBF80E00E94C91400D000D0ADB7BEB731
:102BA0001296DC93CE9311978DE497E014969C9344
:102BB0008E9313970E94DA2C0F900F900F900F9026
:102BC00080919306893080F111E0CE01FC2E092F0F
:102BD000CEE2D7E01CC000D000D000D0EDB7FEB7E9
:102BE0003196ADB7BEB71196FC92119712960C9321
:102BF000D383C283358324830E94DA2C1F5FEDB711
:102C0000FEB736960FB6F894FEBF0FBEEDBF212F6C
:102C100030E08091930690E0019768E070E00E94B8
:102C20002D4F62177307BCF6DF91CF911F910F9163
:102C3000FF9008952F923F924F925F926F927F92F2
:102C40008F929F92AF92BF92CF92DF92EF92FF92BC
:102C50000F931F93DF93CF9300D0CDB7DEB78C01D6
:102C60000D5F1F4FC8010E9422340E94D5365B01C0
:102C70006C010E94A1352C01C601B5010E94AA3544
:102C80003C01C601B5010E94B6354C01C601B50133
:102C90000E94C2359A838983C601B5010E94BC3562
:102CA0001C01C80166E576E040E325E131E00E94C1
:102CB000D633882361F086E596E00E9432064C0107
:102CC000009729F4C601B5010E94B6354C01C80130
:102CD00066E576E040E327E131E00E94D6338823C1
:102CE00029F086E596E00E9432063C01C80166E5BF
:102CF00076E040E329E131E00E94D633882329F0D1
:102D000086E596E00E9432062C012DB73EB72C5185
:102D100030400FB6F8943EBF0FBE2DBF0DB71EB7A3
:102D20000F5F1F4F37E8E32E36E0F32EADB7BEB787
:102D30001296FC92EE92119781E295E0F80193834E
:102D4000828380E790E0958384838091FF0186836E
:102D500017828091090280871186809122028287E2
:102D60001386809104028487158680910E028687DF
:102D7000178680911302808B118AC601B50120E865
:102D800031E541E050E00E94404FD80153963C931A
:102D90002E9352978CE390E0E981FA819C01E29FA7
:102DA000C001E39F900DF29F900D1124820D931DA1
:102DB00055969C938E93549757969C928E925697C5
:102DC00059967C926E9258975B965C924E925A9767
:102DD0000E94DA2C4DB75EB7485E5F4F0FB6F8948D
:102DE0005EBF0FBE4DBFADB7BEB71296FC92EE925E
:102DF000119785E195E014969C938E9313970E940A
:102E0000DA2C00E00F900F900F900F90BE2CEF2C5B
:102E100021E1C22E25E0D22E21C000D000D000D06A
:102E2000EDB7FEB73196ADB7BEB71196BC9211970C
:102E30001296EC92D382C282A02FB0E0A856B44F73
:102E40008C91848315820E94DA2C0F5FEDB7FEB758
:102E500036960FB6F894FEBF0FBEEDBF8091900B73
:102E600097E8892E96E0992E0817B8F200D000D086
:102E7000ADB7BEB712969C928E9211978DE095E0F9
:102E800014969C938E9313970E94DA2C0F900F90B8
:102E90000F900F900E94931500D000D0EDB7FEB7B1
:102EA000928281828EEE94E0948383830E94DA2C56
:102EB000ADB7BEB712969C928E92119789EC94E0B2
:102EC00014969C938E9313970E94DA2C0F900F9078
:102ED0000F900F9081E00F900F90CF91DF911F9195
:102EE0000F91FF90EF90DF90CF90BF90AF909F90A9
:102EF0008F907F906F905F904F903F902F900895AC
:102F00000F931F938DB79EB708970FB6F8949EBF87
:102F10000FBE8DBFEDB7FEB7319607E816E0ADB72F
:102F2000BEB712961C930E93119780E996E0938397
:102F3000828380E790E0958384838FEA90E0978393
:102F400086830E94DA2CEDB7FEB738960FB6F89458
:102F5000FEBF0FBEEDBF0E94931500D000D0ADB7ED
:102F6000BEB712961C930E93119781E796E01496C4
:102F70009C938E9313970E94DA2CEDB7FEB71283C1
:102F800001838CE496E0948383830E94DA2C0F9073
:102F90000F900F900F9081E01F910F9108950F9364
:102FA0001F938C0102960E942234D80112960C9134
:102FB000112707FD10950053104043E0000F111F2B
:102FC0004A95E1F700D000D000D0EDB7FEB73196BA
:102FD00087E896E0ADB7BEB712969C938E93119793
:102FE00087E897E09383828380E790E095838483EA
:102FF0000E94DA2CEDB7FEB736960FB6F894FEBFF6
:103000000FBEEDBF802F0E94C91481E01F910F9168
:103010000895DF92EF92FF920F931F93DF93CF9368
:10302000CDB7DEB761970FB6F894DEBF0FBECDBF48
:1030300020919306821708F043C0222309F440C070
:1030400090E001968C0164E0000F111F6A95E1F792
:10305000080F191F08521C4F51E1D52E7E0108940C
:10306000E11CF11C13C0C701B80141E150E021E2AD
:1030700037E00E948B06C8014197B70141E150E05B
:1030800029E237E00E94A7060F5E1F4F20919306AA
:103090002D9DC001112488529C4F0817190718F361
:1030A000215020939306F999FECF1FBA86ED93E045
:1030B00092BD81BD20BD0FB6F894FA9AF99A0FBE61
:1030C00061960FB6F894DEBF0FBECDBFCF91DF91F2
:1030D0001F910F91FF90EF90DF900895CF93DF93B2
:1030E000EC012396CE010E942234CE010E94AF1043
:1030F000882309F450C0CE0166E576E040E321E183
:1031000031E00E94D633882309F445C086E596E075
:103110000E9432069C018FEF2F3F380781F41092F6
:103120009306F999FECF1FBA86ED93E092BD81BD5B
:1031300010BC0FB6F894FA9AF99A0FBE09C08091A4
:10314000930690E02817390734F5822F0E9409185A
:1031500000D000D000D0EDB7FEB7319687E896E0FA
:10316000ADB7BEB712969C938E93119782E895E007
:103170009383828380E790E0958384830E94DA2C96
:1031800081E02DB73EB72A5F3F4F0FB6F8943EBFA0
:103190000FBE2DBF01C080E0DF91CF910895982F21
:1031A00080919306981760F481E1989FC0011124E3
:1031B00088529C4F41E150E029E237E00E94A70687
:1031C0000895BC01909193069E33F0F481E1989F9D
:1031D000C001112488529C4F41E150E029E237E0C0
:1031E0000E94A706209193062F5F20939306F999DA
:1031F000FECF1FBA86ED93E092BD81BD20BD0FB614
:10320000F894FA9AF99A0FBE0895BF92CF92DF927E
:10321000EF92FF920F931F93DF93CF93CDB7DEB75B
:1032200063970FB6F894DEBF0FBECDBF7C018C0153
:103230000D5F1F4FC8010E942234C8010E94AF10C9
:10324000882309F403C1C80166E576E040E321E183
:1032500031E00E94D633882309F4F8C086E596E071
:103260000E9432066C012FEF8F3F92070CF4EEC0E4
:103270008091930690E0C816D9060CF0E7C01A8337
:10328000098387E690E0E80EF91E0DC0C8016BE1E6
:1032900071E043E050E00E947D06009779F00F5FF7
:1032A0001F4F1A83098309811A81D8018C918823C1
:1032B00009F4CCC00E151F0548F3C8C00D5F1F4FA1
:1032C0001A8309838E010F5F1F4FC8010E94EE0908
:1032D0008B8BC8010E94EE098B83C8010E94EE0906
:1032E0008C83C8010E94EE099E838D83C8010E94D1
:1032F000EE0998878F83C8010E94EE099A87898713
:10330000C8010E94EE099C878B87FF24B02EE12E16
:103310008E01035F1F4F09C08B2D9E2D0E94EE0969
:10332000F801EF0DF11D8083F3948091900BF81656
:1033300098F306C0FC01EF0DF11D1082F39402C05A
:10334000CE010D96B5E0BF15A8F78C81823020F034
:10335000CE0103960E94820D00D000D000D0EDB7C0
:10336000FEB7319607E816E0ADB7BEB712961C93CC
:103370000E9311978EEB94E09383828380E790E025
:10338000958384830E94DA2CEDB7FEB736960FB68C
:10339000F894FEBF0FBEEDBFBE016D5F7F4FFFEF24
:1033A000CF16FFEFDF06C1F4CB010E94E11800D079
:1033B00000D0ADB7BEB712961C930E93119781EA59
:1033C00094E014969C938E9313970E94DA2C0F909E
:1033D0000F900F900F9022C08C2D0E94CF1800D01C
:1033E00000D000D0EDB7FEB73196ADB7BEB712969C
:1033F0001C930E93119783E894E09383828308943F
:10340000C11CD11CD582C4820E94DA2CEDB7FEB754
:1034100036960FB6F894FEBF0FBEEDBF00D000D0B9
:1034200087E896E0ADB7BEB712969C938E9311973E
:1034300082E694E014969C938E9313970E94DA2C64
:1034400081E00F900F900F900F9001C080E0639685
:103450000FB6F894DEBF0FBECDBFCF91DF911F91A5
:103460000F91FF90EF90DF90CF90BF9008950E9452
:10347000E93B0E941640ACE1B8E080E090E0FC013E
:10348000E456F94F1082118212821382FC01E45A31
:10349000F84F10821182128213821D920496803C92
:1034A000910569F708950F931F93CF93DF93EC0174
:1034B0002396CE010E94AF10882309F4E7C0CE0105
:1034C00066E576E040E32FE131E00E94D6338823C1
:1034D00011F00E94371ACE0166E576E040E323E260
:1034E00031E00E94D633882309F44AC086E596E08D
:1034F0000E943206181619060CF042C02DB73EB7CE
:10350000285030400FB6F8943EBF0FBE2DBFEDB728
:10351000FEB7319607E816E0ADB7BEB712961C931A
:103520000E93119788EB92E09383828380E790E07B
:10353000958384838AE090E0978386830E94DA2CC7
:103540000F900F900F900F90EDB7FEB7128301838D
:103550008BEA92E0948383830E94DA2C0F900F9081
:103560000F900F9080918D0690918E0620918B0682
:1035700030918C06821B930B0E94C52F0E94593BF1
:10358000CE0166E576E040E327E231E00E94D633E3
:10359000882399F080915606813339F480918E0BFF
:1035A00080FD0BC00E94A04008C0803331F48091A0
:1035B0008E0B80FF02C00E949640CE0166E576E049
:1035C00040E32AE231E00E94D6338823D9F080918B
:1035D0005606813351F480918E0B84FD13C00E94F6
:1035E000371A80918E0B80610BC0803359F4809123
:1035F0008E0B84FF07C00E94371A80918E0B8F7E3E
:1036000080938E0BCE0166E576E040E32DE231E05B
:103610000E94D633882371F086E596E00E94320638
:10362000181619061CF40E94674004C0892B71F516
:103630000E945F402DB73EB7285030400FB6F89437
:103640003EBF0FBE2DBFEDB7FEB7319687E896E0BF
:10365000ADB7BEB712969C938E9311978EE992E008
:103660009383828380E790E0958384838AE291E06C
:10367000978386830E94DA2C81E0EDB7FEB73896F7
:103680000FB6F894FEBF0FBEEDBF01C080E0DF9122
:10369000CF911F910F910895BF92CF92DF92EF9239
:1036A000FF920F931F93DF93CF9300D0CDB7DEB778
:1036B0007C018C010D5F1F4FC8010E942234C8019C
:1036C0000E94AF10882309F4A0C01A83098327E65B
:1036D00030E0E20EF31E0DC0C80160E371E043E08C
:1036E00050E00E947D06009779F00F5F1F4F1A830C
:1036F000098309811A81D8018C91882309F485C036
:103700000E151F0548F381C00D5F1F4F1A830983F3
:103710000E94371AFF2400E713E0EE246E0108949C
:10372000C11CD11CEEEFBE2E37C0C6010E94EE09AF
:10373000F999FECF1FBA12BD01BD90BD0FB6F89426
:10374000FA9AF99A0FBEF999FECF1FBA0F5F1F4F71
:1037500012BD01BD0150104080BD0FB6F894FA9A19
:10376000F99A0FBE0097A9F02F2D30E0F901EE0F66
:10377000FF1FEE0FFF1FE45AF84FA0E0B0E0808378
:103780009183A283B383245E374FF901B082EE2484
:10379000E394F3940E5F1F4F8091910BF81608F499
:1037A000C4CFEE2031F00E94D5364091FF010E9437
:1037B0003F072DB73EB7285030400FB6F8943EBFB4
:1037C0000FBE2DBFEDB7FEB7319687E896E0ADB7D7
:1037D000BEB712969C938E9311978DE996E09383D2
:1037E000828380E790E0958384838AE291E09783E7
:1037F00086830E94DA2C81E0EDB7FEB738960FB6CB
:10380000F894FEBF0FBEEDBF01C080E00F900F9097
:10381000CF91DF911F910F91FF90EF90DF90CF90AC
:10382000BF900895EF92FF920F931F939B01AC01FD
:1038300080914C0890914D08A0914E08B0914F088E
:103840000097A105B10549F420934C0830934D0829
:1038500040934E0850934F0854C079018A01E81AEA
:10386000F90A0A0B1B0BD801C701CD97A105B105B9
:1038700008F447C020934C0830934D0840934E08FD
:1038800050934F0886E09BE00E94FA300E94CD4A98
:103890007B018C010E943C380E94473186E09BE00E
:1038A0000E94BB33882361F40E94CD4A6E197F09C0
:1038B000800B910B683C71058105910558F319C087
:1038C00080918F0B8F7080938F0B80918F0B8295DF
:1038D0008F7090E00397ACF08091F501882389F018
:1038E0006091D0027091D10287E491E00E9463431D
:1038F00008C080918F0B982F907F905F8F70892BDD
:10390000E2CF1F910F91FF90EF900895EF92FF92F9
:103910000F931F939B01AC018091B9018823C9F1DA
:1039200080918F0B82958F70A1F580918F06909179
:103930009006A0919106B09192060097A105B1055D
:1039400069F079018A01E81AF90A0A0B1B0BD80100
:10395000C70181589145A140B040D8F020938F060F
:103960003093900640939106509392060E94AE09C0
:103970007B018C01611571058105910551F00E9453
:10398000A83680918E0B85FF04C0C801B7010E9444
:10399000BF3A1F910F91FF90EF9008950E947E42D1
:1039A0000E94FC400E94E8079091F00180E0209185
:1039B000EB01820F911D9093D1028093D0026CE3B2
:1039C00070E080E090E00E949F3680918E0B85FD34
:1039D00003C080E090E002C088EE9AE30E9448377E
:1039E00064EF71E080E090E00E94DB4A80E00E949A
:1039F000344280E798E061E00E94753D8AE598E0F6
:103A000060E00E94F925882329F480918E0B806460
:103A100080938E0B82E698E061E00E94753D609194
:103A2000D0027091D10287E491E00E946343882321
:103A300021F080918F0B8F7004C080918F0B8F705D
:103A4000806180938F0B64EF71E080E090E00E94D2
:103A5000DB4A0E94164010928F0610929006109238
:103A6000910610929206089582E00E94E63C282F6B
:103A700030E086FF41C02F7030702230310591F068
:103A80002430310509F121303105B1F587FF03C03C
:103A90000E94A04008956091A5017091A6018EEF4B
:103AA0009AE009C087FF03C00E949640089586E00F
:103AB0009BE060E070E00E94CE3F60ED77E080E048
:103AC00090E00E94DB4A089587FF06C081E00E94D3
:103AD000E63C0E94593B089520918F0B822F8F70F6
:103AE00090E06091900B019670E00E942D4F8F70D6
:103AF000207F282B20938F0B08952F923F924F9277
:103B00005F926F927F928F929F92AF92BF92CF926D
:103B1000DF92EF92FF920F931F93DF93CF93CDB776
:103B2000DEB7A9970FB6F894DEBF0FBECDBF2091C8
:103B3000FF012C8B309109023B8B0E943C380E9484
:103B400047319C019093510880935008009799F059
:103B500010928A061092890688E093E090938C0672
:103B600080938B0690938E0680938D06C9018E52AA
:103B70009D4F0E94E90C0E94341D0E94D5364B01D6
:103B80005C018091560890915708A0915808B09117
:103B9000590888159905AA05BB0509F4A3C28092A6
:103BA000560890925708A0925808B092590880E0A1
:103BB0000E94344280918E0B81FF0FC080919E0B3A
:103BC00090919F0BA091A00BB091A10B8816990624
:103BD000AA06BB0610F00E945F400E942F3D809114
:103BE0008E0B84FDC4C083FF04C04C89442309F0BC
:103BF000BEC0C501B4012CE330E040E050E00E94BB
:103C0000404F79018A018091520890915308A09108
:103C10005408B0915508E816F9060A071B0709F47D
:103C2000A6C0E0925208F0925308009354081093F3
:103C30005508662410E09B89892F90E099A788A7F2
:103C40008AC0862DBE016F5F7F4F0E947913CE011F
:103C50000196B501A4010E94C912882309F47AC013
:103C600029853A852115310509F474C0A091900B7E
:103C7000AE8B77241A8A190144245524B62DBF5FD0
:103C8000BFA353C08A898C0DE82EFF24C70101967B
:103C9000E8A5F9A5E817F907E1F1ABA1BCA18C9162
:103CA00090E00C2C02C0959587950A94E2F780FD70
:103CB00030C0EDA1FEA1808190E00C2C02C0959552
:103CC00087950A94E2F780FF24C08701000F111F37
:103CD000000F111F045A184F6091220270E080E01B
:103CE00090E0A20191010E94EE4E24E630E040E017
:103CF00050E00E94404FD8012D933D934D935C932B
:103D00001397ECE1F8E0EE0EFF1EEFA1D701EC9364
:103D100011E00894C11CD11CF8E0CF16D10409F0C1
:103D2000B1CF73942A89285F2A8B3E89731690F449
:103D3000872D90E0CC24DD24AC014E56544F5CA37B
:103D40004BA3ABE0B0E0AC0FBD1FA80FB91FBEA3E3
:103D5000ADA398CF639480919306681608F471CF51
:103D6000112329F0C501B4014C890E943F078091BD
:103D70008E0B83FF4BC13324FB89EF2FF0E0FC8FC8
:103D8000EB8F2B882A94222D30E0C901880F991FD0
:103D9000880F991FAC014456594F5E8F4D8FDC013F
:103DA000A45AB84FB8A3AF8FF901E45EF74FFAA356
:103DB000E9A30FC1832D90E0FC01EE56F44F208162
:103DC000F32DFF0FFF0FFF0FFD8B66247724422F8B
:103DD00050E0588F4F8BDC01A856B44FBA8FA98F93
:103DE000FD88F60C8F89988D062C02C095958795D5
:103DF0000A94E2F7CF2CDD2480FF53C08601000F28
:103E0000111F000F111FF801E45AF84F80819181B2
:103E1000A281B38188169906AA06BB0608F4D0C011
:103E20008F2D60E00E94C53BC6010196EB8DFC8D95
:103E3000E817F907E1F0F0929406F601E45EF74F17
:103E40008081809395060456194FD8018D919C91DD
:103E5000F401E81BF90BF0939706E0939606809225
:103E6000980690929906A0929A06B0929B06F60147
:103E7000EE0FFF1FEE0FFF1FDF01A456B94F1D927B
:103E80001D921D921C921397E45AF84F10821182D2
:103E9000128213822CE138E0C20ED31ED6011C928E
:103EA0008FC09601220F331F220F331F8901045642
:103EB000194FF80180819181A281B38188169906FA
:103EC000AA06BB0608F47CC0ACE54A2EA7E05A2E31
:103ED000420E531EF20180819181A281B381881626
:103EE0009906AA06BB0608F06BC08F2D61E00E9400
:103EF000C53BFB89FF2309F463C0C60101962B8DE6
:103F00003C8D2817390709F45BC0A98DBA8D8C91B7
:103F100090E0062C02C0959587950A94E2F780FF01
:103F20004FC0BC89BB2309F44BC080918E0B84FD2C
:103F300047C080910E02F801208131814281538176
:103F4000280F311D411D511DAD8DBE8D2D933D930B
:103F50004D935C93139780911302E82EFF2400E0A9
:103F600010E084EC9FEFAFEFBFEFE80EF91E0A1FE1
:103F70001B1FF20180819181A281B381E80EF91E9D
:103F80000A1F1B1FAF8DB8A1ED92FD920D931C93DC
:103F90001397ECE1F8E0CE0EDF1ED6018C91E9A17B
:103FA000FAA1808382169306A406B50648F08E1403
:103FB0009F04A006B10620F4822D61E00E94C53B5B
:103FC0000894611C711CF8E06F16710409F008CFA9
:103FD00033948091900B381608F4ECCE0E94164072
:103FE0003091910BECE5F7E020E00DC081919191CB
:103FF000A191B1910197A109B1098E5F9F4FAF4F78
:10400000BF4F20F02F5F231788F361C05B895523D2
:1040100069F080918E0B84FF09C01091910B40E0F4
:1040200021E030E08B89682F70E02EC09C899923B5
:10403000A1F331C0842F90E06217730711F1DC0106
:10404000F3E0B695A795FA95E1F7542F5770FD0167
:10405000EE56F44F808190E0052E02C0959587952D
:104060000A94E2F780FF0DC0A856B44F8C9190E0FF
:1040700002C0959587955A95E2F780FF02C061E0EE
:1040800006C04F5F2F5F3F4F4117A0F260E08B8962
:1040900081500E94C53B0E941640C501B40123E037
:1040A00030E040E050E00E94404F9B01AC012C58B2
:1040B0003D4F81E0D9016C910E94463FC501B4019A
:1040C0000E94121CC501B4010E94861C0BC00E94F4
:1040D000E93B80918E0B877F80938E0BB091090214
:1040E000BB8B94CFA9960FB6F894DEBF0FBECDBFA1
:1040F000CF91DF911F910F91FF90EF90DF90CF90C4
:10410000BF90AF909F908F907F906F905F904F90F7
:104110003F902F900895FC01EF5BFD4F1082779642
:10412000108208951092B50A0895FC01E55AFD4FDA
:104130008081882319F4862F0E942A2A0895EF92FD
:10414000FF920F931F937C018B01472F5527FC0192
:10415000858D968D480F591F60E070E0C7018F5B19
:104160009F4F0E94C82A1070000F111F0E0D1F1DB7
:104170000E5B1F4FF801308120E08291280F311D26
:10418000C9011F910F91FF90EF9008958F929F9218
:10419000AF92BF92CF92DF92EF92FF920F931F9355
:1041A000CF93DF93EC01C85ADD4F8881C855D240C8
:1041B000813009F0C4C0CC5ADD4FE880F9800A8113
:1041C0001B81C455D240E114F1040105110559F4D5
:1041D000C25BDD4F88819981CE54D240892B19F47E
:1041E0006DEF7FEFB3C0298530E040E050E0C801BB
:1041F000B7010E94404F611571058105910589F451
:10420000E114F1040105110561F08E01025B1D4FFF
:10421000F80160817181CE010E949F20F801918395
:104220008083A984BB24CC24DD24EA84FB8400E0C1
:1042300010E08D899E89AF89B88DE80EF91E0A1F9E
:104240001B1F6B897C8980E090E02C8530E040E08A
:1042500050E00E94EE4EE60EF71E081F191FF4E50F
:104260008F2EF2E09F2E8C0E9D1EF40160817181D5
:1042700082819381A60195010E94404FE60EF71EB0
:10428000081F191F8D859E85A0E0B0E0E4E0B6957B
:10429000A79597958795EA95D1F7E80EF91E0A1F1D
:1042A0001B1FC25BDD4F68817981CE54D24080E014
:1042B00090E06250704080409040A60195010E94BD
:1042C000EE4EE60EF71E081F191FCE018F5B9F4FA3
:1042D000B801A7010E94C82A882319F0682F70E04E
:1042E00035C0F4012081318142815381DA01C90155
:1042F0000196A11DB11D80839183A283B383C05B0E
:10430000DD4FE880F9800A811B8179E0880F991FD1
:10431000AA1FBB1F7A95D1F7E816F9060A071B07F3
:1043200018F060E072E012C069E0220F331F441FF2
:10433000551F6A95D1F7B701621B730B07C088231D
:1043400019F061EF7FEF02C060EF7FEFCB01DF91EB
:10435000CF911F910F91FF90EF90DF90CF90BF9082
:10436000AF909F908F9008954F925F926F927F923F
:104370008F929F92AF92BF92CF92DF92EF92FF9275
:104380000F931F93CF93DF934C013B018DE390E09C
:10439000880E991EE401E880F9800A811B81E3EC14
:1043A000FFEF8E0E9F1E49E5442E42E0542E480C2E
:1043B000591CE2018881998135E0880F991F3A954F
:1043C000E1F7AC01452F5527469520E03EEF429F8F
:1043D000E001439FD00D529FD00D1124C80FD91F6B
:1043E0005A01CC24DD24AE0CBF1CC01ED11E84019A
:1043F0000F5B1F4FC801B601A5010E94C82A17C054
:10440000A096F20180819181019691838083F2E0F0
:10441000C030DF0761F40894A11CB11CC11CD11C81
:10442000C801B601A5010E94C82AC0E0D0E0F4018D
:10443000EC0FFD1FEF5BFF4F8081882309F49DC0C7
:10444000DE011B96F401EA0FFB1FEF5BFF4F80813B
:104450008871B1F6F401EC0FFD1FEF5BFF4F808117
:10446000853E71F2CF5BDF4FA4014C0F5D1FC1543D
:10447000D04020E030E0B301620F731FFA01819158
:10448000AF01FB0180832F5F3F4F2830310599F743
:104490002896F401EC0FFD1F9E0128503040EF5B81
:1044A000FF4F8191E301898781918A8780818B8782
:1044B00018861C86A80DB91DAF5BBF4F8C918D87E8
:1044C000280D391D205B3F4FF901908180E0E90103
:1044D0004A919E01840F911DF301978786872D5F76
:1044E0003F4FE901988180E0F90142919F01840FDB
:1044F000911DE301998B888B255F3F4FF9019081D6
:1045000080E0E9014A919E01840F911DF301938B94
:10451000828B2B5F3F4FE901488150E060E070E003
:10452000742F662755274427F901829190E0A0E077
:10453000B0E0DC0199278827482B592B6A2B7B2B6D
:10454000EF019A9180E0FE01229130E0822B932BC3
:10455000A0E0B0E0482B592B6A2B7B2BF301448B56
:10456000558B668B778BF401E75AFD4F80819181E3
:1045700001969183808380E001C081E0DF91CF913B
:104580001F910F91FF90EF90DF90CF90BF90AF9071
:104590009F908F907F906F905F904F9008956F9253
:1045A0007F928F929F92AF92BF92CF92DF92EF92C3
:1045B000FF920F931F93CF93DF93EC016B01ED9666
:1045C000E880F9800A811B81ED9789E5A82E82E0B9
:1045D000B82EAC0EBD1ED5011D921C92B1E48B2EDF
:1045E000912C8C0E9D1EC401B801A7010E94C82AFF
:1045F000F4018081882309F4D8C020E030E022C093
:10460000205E3F4FD5018D919C91119701968D931E
:104610009C93B2E020303B0761F40894E11CF11C4C
:10462000011D111DC401B801A7010E94C82A20E084
:1046300030E0FE01E20FF31FEF5BFF4F8081882324
:1046400009F4B3C0ABE06A2E712C620E731EFE013A
:10465000E60DF71DEF5BFF4F8081887189F6FE0143
:10466000E20FF31FEF5BFF4F8081853E49F22F5B26
:104670003F4FBE01620F731F2154304040E050E0B5
:104680008601040F151FFB018191BF01D8018C9396
:104690004F5F5F4F4830510599F7285F3F4FFE014C
:1046A000E20FF31F28503040EF5BFF4F8191D6019E
:1046B00019968C93199781911A968C931A978081E9
:1046C0001B968C931B9718961C9218971C961C92FD
:1046D0006C0E7D1EE1E4F0E06E0E7F1ED3018C9126
:1046E000F60185872C0F3D1F205B3F4FD9019C9120
:1046F00080E0F90142919F01840F911DD6011F9620
:104700009C938E931E972D5F3F4FF901908180E01F
:10471000D9014E919D01840F911DF601918B808BE3
:10472000255F3F4FD9019C9180E0F90142919F01A3
:10473000840F911DD60153969C938E9352972B5FB5
:104740003F4FF901408150E060E070E0742F662730
:1047500055274427D9018E919D0190E0A0E0B0E05B
:10476000DC0199278827482B592B6A2B7B2BF901D1
:10477000929180E0229130E0822B932BA0E0B0E078
:10478000482B592B6A2B7B2BD60154964D935D9366
:104790006D937C935797FE01E75AFD4F808191817D
:1047A00001969183808380E001C081E0DF91CF9109
:1047B0001F910F91FF90EF90DF90CF90BF90AF903F
:1047C0009F908F907F906F9008956F927F928F92BD
:1047D0009F92AF92BF92CF92DF92EF92FF920F9390
:1047E0001F93DF93CF93CDB7DEB7A5970FB6F8949D
:1047F000DEBF0FBECDBF7C016B01AB0120E030E01E
:104800000CC0FA019081892F81568A3108F49052A8
:10481000FA019193AF012F5F3F4FF6010190002005
:10482000E9F73197EC19FD092E173F0750F38E0178
:10483000025F1F4FC701B8010E94CF22F82EF1E09E
:104840008F1709F490C040E050E0B8019E012F5F3F
:104850003F4F06C0F901E40FF51F80834F5F5F4FA4
:10486000FB01E40FF51F8081803219F048305105BB
:1048700089F7CE010196FC01E40FF51F2EE220839B
:10488000DA01119647E1642E712C6C0E7D1E8A0FA1
:104890009B1FB301AE01455E5F4F04C0FC01219335
:1048A000CF011196FB012081203229F06F5F7F4FED
:1048B0006417750799F78E010F5F1F4FA00FB11F87
:1048C0001C92C801B6010E946D060097E9F54DC023
:1048D0008AE598E0B5010E94B421F82E882309F0FA
:1048E0003FC080E090E005C0F801E80FF91F208389
:1048F0000196F501E80FF91F2081203219F0883068
:10490000910591F7F801E80FF91FE082DC0111969B
:10491000C8018A0F9B1FA30104C0FC012193CF0192
:104920001196FA012081203229F04F5F5F4F481520
:10493000590599F7A00FB11F1C92C801B6010E943A
:104940006D06009729F611C03EE0A32EB12CAC0EE7
:10495000BD1E2EE2E22E9BE1892E912C8C0E9D1E17
:10496000FF2009F4B5CF80E001C081E0A5960FB625
:10497000F894DEBF0FBECDBFCF91DF911F910F9195
:10498000FF90EF90DF90CF90BF90AF909F908F906F
:104990007F906F9008953F924F925F926F927F92B7
:1049A0008F929F92AF92BF92CF92DF92EF92FF923F
:1049B0000F931F93DF93CF93CDB7DEB7A5970FB6B5
:1049C000F894DEBF0FBECDBF8C01B62EC72E342E9D
:1049D0000F5B1D4FF801808101541240882311F0B4
:1049E00081E1EFC0862F972F9C01A90120E030E0E4
:1049F0000CC0FA019081892F81568A3108F49052B7
:104A0000FA019193AF012F5F3F4FAB2DBC2DFD01FC
:104A100001900020E9F73197EA1BFB0B2E173F07A7
:104A200040F33EE0E32EF12CEC0EFD1EC801B70171
:104A30000E94CF22D82EF1E08F1709F4C1C040E0C8
:104A400050E0B7019E012F5F3F4F06C0F901E40F10
:104A5000F51F80834F5F5F4FFB01E40FF51F8081DF
:104A6000803219F04830510589F7CE010196FC01DA
:104A7000E40FF51F2EE22083DA01119627E1422E82
:104A8000512C4C0E5D1E8A0F9B1FB201AE01455E7C
:104A90005F4F04C0FC012193CF011196FB012081DF
:104AA000203229F06F5F7F4F6417750799F77E01F9
:104AB0000894E11CF11CAE0DBF1D1C92C7016B2DAB
:104AC0007C2D0E946D06009709F06BC0F701D8019C
:104AD000AF5BBD4F9E01225F3F4F81918D93E217E7
:104AE000F307D9F748C08AE598E0B4010E94B421E1
:104AF000D82E882309F061C080E090E005C0F7015E
:104B0000E80FF91F20830196F401E80FF91F2081B7
:104B1000203219F08830910591F7F701E80FF91F5D
:104B2000A082DC011196C7018A0F9B1FA20104C05D
:104B3000FC012193CF011196FA012081203229F046
:104B40004F5F5F4F4615570599F7AE0DBF1D1C927D
:104B5000C7016B2D7C2D0E946D06009721F6F70191
:104B6000D801AF5BBD4F9E01225F3F4F81918D9376
:104B7000E217F307D9F7025B1D4F88A199A1F8014D
:104B8000819391938AA19BA1ACA1BDA181939193A3
:104B9000A193B1931192119211921192308280E0FF
:104BA00010C0AEE08A2E912C8C0E9D1EFEE2AF2E20
:104BB000EBE16E2E712C6C0E7D1EDD2009F493CF7F
:104BC00080E1A5960FB6F894DEBF0FBECDBFCF91A2
:104BD000DF911F910F91FF90EF90DF90CF90BF90EA
:104BE000AF909F908F907F906F905F904F903F908D
:104BF00008950F931F93CF93DF93EC01862F0E94AC
:104C0000302B8E010F5B1F4FC80140E050E060E089
:104C100070E00E94C82A882311F080EF84C1C15C33
:104C2000DD4F8881CF53D240853509F079C1C05C12
:104C3000DD4F8881C054D2408A3A09F071C1CD5FFE
:104C4000DD4F7881C350D2407883C65FDD4F288125
:104C500030E040E050E0522F4427332722278A914A
:104C600090E0A0E0B0E0DC0199278827280F391FE9
:104C70004A1F5B1F9A9180E06A91C750D240860F0D
:104C8000911DA0E0B0E0280F391F4A1F5B1F298348
:104C90003A834B835C83C25FDD4F288130E040E084
:104CA00050E0522F4427332722278A9190E0A0E03A
:104CB000B0E0DC0199278827280F391F4A1F5B1FA6
:104CC0009A9180E06A91CB50D240860F911DA0E06E
:104CD000B0E0280F391F4A1F5B1F2D833E834F838F
:104CE0005887743031F0763021F0763811F082EF49
:104CF0001AC149815A816B817C81C8010E94C82AEE
:104D0000882311F080EE0FC1C15CDD4F8881CF5345
:104D1000D240853509F006C1C05CDD4F8881C054A2
:104D2000D2408A3A09F0FEC0C25BDF4F8881CE5480
:104D3000D0408987C05BDF4F988180E02A91CF54B3
:104D4000D040820F911D9B878A87CF5ADF4F888181
:104D5000C155D0408C87CD5ADF4F988180E02A9191
:104D6000C255D040820F911D9E878D87CB5ADF4F51
:104D7000988180E02A91C455D040820F911DA0E017
:104D8000B0E08F87988BA98BBA8B0097A105B105EE
:104D900031F5CC59DF4F288130E040E050E0522F10
:104DA0004427332722278A9190E0A0E0B0E0DC017D
:104DB00099278827280F391F4A1F5B1F9A9180E087
:104DC0006A91C156D040860F911DA0E0B0E0280F37
:104DD000391F4A1F5B1F2F87388B498B5A8BC85A44
:104DE000DF4F788160E08A91C755D040680F711D10
:104DF0007C8B6B8BC05ADF4F288130E040E050E065
:104E0000522F4427332722278A9190E0A0E0B0E078
:104E1000DC0199278827280F391F4A1F5B1F9A91A9
:104E200080E0EA91CD55D0408E0F911DA0E0B0E01A
:104E3000280F391F4A1F5B1F2D8B3E8B4F8B588FBE
:104E4000C559DF4F288130E040E050E0522F442721
:104E5000332722278A9190E0A0E0B0E0DC01992777
:104E60008827280F391F4A1F5B1F9A9180E0EA911B
:104E7000C856D0408E0F911DA0E0B0E0280F391F1A
:104E80004A1F5B1F298F3A8F4B8F5C8FEA85FB850A
:104E90009F0140E050E089819A81AB81BC81280F5D
:104EA000391F4A1F5B1F8C8590E0DC01A69FC00163
:104EB000A79F900DB69F900D1124A0E0B0E0280FA1
:104EC000391F4A1F5B1FED96288339834A835B8312
:104ED000ED9789819A818E0F9F1F9E8F8D8F860FF0
:104EE000971F98A38F8F6D817E818F81988549E070
:104EF000660F771F881F991F4A95D1F70E94FD4DB5
:104F000020E030E040E855E30E948B4E69A37AA38D
:104F10008BA39CA3C55ADD4F81E0888380E003C04A
:104F200081EF01C081EEDF91CF911F910F91089524
:104F3000DF93CF9300D000D000D0CDB7DEB7DE0135
:104F40001196E7E7F2E086E001900D928150E1F7DB
:104F500086E191E0E2EDF2E0DF019C011D9221503B
:104F60003040E1F78091B60A833019F46AE07BE0C3
:104F700003C0BE016F5F7F4F84E490E043E450E0E4
:104F80000E94832E8091B60A833039F082ED92E040
:104F9000BE016F5F7F4F0E94653481E08093FC0209
:104FA0008093FD0286E08093FE028091C30A909177
:104FB000C40AA091C50AB091C60A809300039093D9
:104FC0000103A0930203B09303038091B60A8330D8
:104FD00039F48CEF92E00C966EEF7AE00E946D341B
:104FE00088E193E068EF7AE00E946534A8EEB3E0D0
:104FF000EBE9F1E002C081918D9331E0E13AF307F2
:10500000D1F79091B60A992311F083E001C081E0B5
:105010008093EE038DE38093EF0387E08093F003AA
:1050200081E08093F103A2EFB3E0E8EFFAE002C081
:1050300081918D938AE0EE3FF807D1F78CE0809361
:10504000F8038AE08093F903EAE8F1E0AAEFB3E01D
:1050500002C081918D9321E0E439F207D1F724E079
:1050600034E03093C80A2093C70A913069F582E38F
:105070008093040484E080930504D9011296EEEF36
:10508000FAE002C081918D933BE0E230F307D1F763
:1050900086E380930A0484E080930B048CE094E020
:1050A0009093C80A8093C70ADC01EAE0FBE002C0E3
:1050B00081918D938BE0EE30F807D1F780E194E099
:1050C0009093C80A8093C70A2091C70A3091C80AF2
:1050D000D901E5E9F1E002C081918D9381E0EB39DE
:1050E000F807D1F7C90106969093C80A8093C70ABA
:1050F0008C5F92400E947A3026960FB6F894DEBFFD
:105100000FBECDBFCF91DF910895DF92EF92FF9256
:105110000F931F93CF93DF938C018091B60A823057
:1051200009F4F7C0833030F4882351F1813009F05D
:1051300054C14AC0833021F0843009F04EC1E9C027
:105140000E94CD4A2091BB0A3091BC0A4091BD0A11
:105150005091BE0AE090B70AF090B80A0091B90ADF
:105160001091BA0A2E0D3F1D401F511F6217730781
:105170008407950708F431C10E94982784E017C07E
:105180000E94CD4A6093C30A7093C40A8093C50AF3
:105190009093C60A1092FE0A1092FF0A1092000B1A
:1051A0001092010B0E9498270E94CC3781E08093D7
:1051B000B60A0E94CD4A6093BF0A7093C00A8093DA
:1051C000C10A9093C20A09C10634110508F4F0C05F
:1051D0008091F502833409F0EBC0209100033091F7
:1051E000010340910203509103038091C30A9091FF
:1051F000C40AA091C50AB091C60A281739074A0700
:105200005B0709F0D5C0CCEED3E0FE01A8014E52F9
:105210005D4FDF01119691819D012F5F3F4F80818E
:10522000853321F411968C91823039F0F901E90F20
:10523000F11DE417F50768F3BBC08EEF9AE06CE050
:1052400073E00E946D3452EDE52E52E0F52EE00E33
:10525000F11EFE013196D9808F010F5F1F4F8881AB
:105260008630A9F0873030F4813059F0833009F06E
:1052700045C00AC08633E9F18A3361F08333F1F522
:1052800009C082E09BE037C086E09BE034C08EE03E
:105290009BE031C0618170E080E090E0982F872F23
:1052A000762F6627F8012181620F711D811D911DE6
:1052B000982F872F762F66272281620F711D811DFF
:1052C000911D982F872F762F66272381620F711DDE
:1052D000811D911D28EE33E040E050E00E94EE4E2B
:1052E0006093BB0A7093BC0A8093BD0A9093BE0A78
:1052F00005C08AE09BE0B8010E946D34E801CD0D45
:10530000D11DCE15DF0508F4A4CF0E94982782E0B6
:105310004ECF0634110508F44BC08091F50283345A
:1053200009F046C02091000330910103409102032F
:10533000509103038091C30A9091C40AA091C50AB9
:10534000B091C60A281739074A075B0789F5ECEEC2
:10535000F3E0A8014E525D4FDF01119691819D014E
:105360002F5F3F4F8081853321F411968C918530DA
:1053700039F0F901E90FF11DE417F50768F318C0DA
:105380000E94C7370E94CD4A6093B70A7093B80A4B
:105390008093B90A9093BA0A8091060B882321F072
:1053A00086E09BE00E94E92E83E08093B60A15C058
:1053B0000E94CD4A2091BF0A3091C00A4091C10A93
:1053C0005091C20A205F384D4F4F5F4F2617370765
:1053D0004807590710F41092B60ADF91CF911F9138
:1053E0000F91FF90EF90DF900895CF93DF9381E0CE
:1053F0008093160B9091FD0A892F82958F70805DA6
:10540000809392019F70905D909393011092B60AE1
:105410000E94CD4AEB0104C00E943C380E948528BE
:105420008091B60A833061F00E94CD4A6C1B7D0BDF
:1054300060567A4E28F40E94FD37882389F3ECCF1A
:1054400090E08091B60A833009F491E0892FDF91D2
:10545000CF9108958093C90A08951F93CF93DF9346
:105460000E94CD4AEB011FEF09C00E94CD4A6C1B80
:105470007D0B6955724010F08FE00CC01EBD0DB45D
:1054800007FEFDCF8EB58F3F81F38E3F11F481E093
:105490000DC08DE08093CB0AE091CC0AF091CD0A4B
:1054A00080819091CE0A892B808380E0DF91CF911B
:1054B0001F910895FF920F931F93CF93DF938C0159
:1054C0000E94CD4AEB01FF24FA94FEBC0DB407FE06
:1054D000FDCF8EB58F3F11F481E008C00E94CD4A08
:1054E0006C1B7D0B6017710780F380E0DF91CF911B
:1054F0001F910F91FF900895DF92EF92FF920F930B
:105500001F93182FD42EE52EF62E072FE091CC0AEC
:10551000F091CD0A90818091CE0A80958923808375
:105520008CE291E00E945A2A812F80648EBD0DB4D6
:1055300007FEFDCF0EBD0DB407FEFDCFFEBC0DB4C2
:1055400007FEFDCFEEBC0DB407FEFDCFDEBC0DB4F3
:1055500007FEFDCF112311F485E905C0183011F4C1
:1055600087E801C08FEF8EBD0DB407FEFDCF90E040
:105570002FEF2EBD0DB407FEFDCF8EB587FF02C005
:105580009150B9F71F910F91FF90EF90DF90089520
:10559000EF92FF920F931F93CF93DF93EC017A0169
:1055A0008B018091CA0A833039F089E0EE0CFF1C30
:1055B000001F111F8A95D1F781E1B801A7010E9450
:1055C0007C2A8823C9F70E942D2A882319F4109277
:1055D000CB0A1BC08FEF8EBD20E030E09FEF0DB4F3
:1055E00007FEFDCF8EB5FE01E20FF31F80839EBD47
:1055F0002F5F3F4F81E02F3F380789F70DB407FE3B
:10560000FDCF8EB5C150DE4F8883E091CC0AF0917A
:10561000CD0A80819091CE0A892B808380E0DF9132
:10562000CF911F910F91FF90EF900895DF92EF922D
:10563000FF920F931F93D82E7A018B0187E340E0EE
:1056400050E060E070E00E947C2A8D2DB801A70137
:105650000E947C2A1F910F91FF90EF90DF90089598
:10566000EF92FF920F931F93CF93DF93082F0E9427
:10567000CD4AEB01E091C90A8E2F90E0FC01EC5578
:10568000F44FE491F0E0EE0FFF1FE057F44F259147
:1056900034913093CD0A2093CC0A8C53944FFC0163
:1056A00074917093CE0AE091A3018E2F90E0FC01DB
:1056B000EC55F44FE491F0E0EE0FFF1FE057F44F8C
:1056C000A591B491B093D00AA093CF0A8C53944F74
:1056D000FC0164916093D10AE091A2014E2F50E049
:1056E000FA01EC55F44FE491F0E0EE0FFF1FE057A4
:1056F000F44F859194919093D30A8093D20A4C539E
:10570000544FFA0184918093D40AE091A4014E2F62
:1057100050E0FA01EC55F44FE4918E2F90E0880FA1
:10572000991F8057944FFC01E590F490F092D60AAF
:10573000E092D50A4C53544FFA0194919093D70AB2
:10574000F9018081872B8083F7018081892B8083F9
:105750008C91862B8C938091C90A61E00E94334919
:105760008091A20161E00E9433498091A40161E02F
:105770000E9433498091A30160E00E9433498091E7
:10578000A10161E00E9433498091A10161E00E9482
:105790007249E091CC0AF091CD0A80819091CE0AB5
:1057A000892B808383E58CBD8DB58E7F8DBD80E098
:1057B0002FEF2EBD0DB407FEFDCF8F5F8A30C9F7E6
:1057C000808190959823908309C00E94CD4A6C1BDC
:1057D0007D0B615D774010F081E048C080E040E0E3
:1057E00050E060E070E00E947C2A182F813069F759
:1057F00088E04AEA51E060E070E00E947C2A82FF83
:1058000003C01093CA0A1BC080E02FEF2EBD0DB459
:1058100007FEFDCF9EB58F5F8430C1F79A3A11F035
:1058200082E024C082E08093CA0A09C00E94CD4A67
:105830006C1B7D0B615D774010F088E017C089E23A
:1058400040E050E060E070E00E94162B882371F782
:105850008091CA0A823071F58AE340E050E060E04E
:1058600070E00E947C2A882379F086E08093CB0A3E
:10587000E091CC0AF091CD0A80819091CE0A892BDB
:1058800080838091CB0A29C08FEF8EBD0DB407FEB7
:10589000FDCF8EB5807C803C19F483E08093CA0AEA
:1058A00080E09FEF9EBD0DB407FEFDCF2EB58F5F4C
:1058B0008330C1F7E091CC0AF091CD0A80819091BC
:1058C000CE0A892B8083073028F086E18093CB0AAB
:1058D00080E003C000650CBD81E0DF91CF911F9196
:1058E0000F91FF90EF9008950F931F93CF93DF9345
:1058F0009C01EB018A011092160B009729F08EEFA4
:105900009AE0B9010E946D34209719F0CE010E94EF
:10591000E92E0115110529F08EE09BE0B8010E94E7
:105920006D3481E0DF91CF911F910F910895AF9277
:10593000BF92CF92DF92FF920F931F93CF93DF938B
:105940008C01EB01F42E1092160B38E341E050E08D
:1059500060E070E018C0832F90E0FC01B3E0F595A3
:10596000E795BA95E1F7E852F54F877090705A01C4
:105970006B0104C0AA0CBB1CCC1CDD1C8A95D2F7A1
:1059800020812A292083315031F788EF9AE0BE0127
:105990000E946534C80168EF7AE04F2D0E942139DA
:1059A000DF91CF911F910F91FF90DF90CF90BF902B
:1059B000AF900895CF92DF92EF92FF920F931F93D3
:1059C000DF93CF93CDB7DEB7EB84FC84CD84DE8448
:1059D000DE011F9601C0D801F6018491882309F4E5
:1059E000BCC00894C11CD11C843209F099C0F601D6
:1059F0000894C11CD11C8491863409F45FC087349B
:105A000034F4843469F0853409F08AC06EC08C3473
:105A1000C9F1833509F445C0883409F081C00DC04F
:105A20008D010E5F1F4FF701668177818D919C91EB
:105A30004AE050E00E94C3067EC02C91822F992735
:105A400087FD909514E0959587951A95E1F78F70ED
:105A50002F702A300CF0295F8A300CF0895F8D019D
:105A60000E5F1F4FF701A681B781805DFD01819315
:105A7000205D11962C933196D7011796FC93EE93E7
:105A80001697A9CF8D010C5F1F4F6D917D918D9160
:105A90009C91F701468157812AE030E00E94EC0694
:105AA0004AC08D010E5F1F4F6D917C91D7011696F4
:105AB0008D919C9117970E9476063DC08D010E5FD7
:105AC0001F4F2D913C910AC0D7011696ED91FC9184
:105AD000179781931796FC93EE931697F9012F5F12
:105AE0003F4F8491882381F776CF8D010E5F1F4F42
:105AF0002D913C910AC0D7011696ED91FC91179714
:105B000081931796FC93EE931697F999FECF32BDC9
:105B100021BDF89A80B52F5F3F4F882361F75BCF97
:105B2000F70126813781F90181939F01F7013783BE
:105B300026838D0150CFD70116968D919C91179792
:105B4000FC0101900020E9F73197E81BF90B8E0F5B
:105B50009F1FF701978386833ECFCF91DF911F91DF
:105B60000F91FF90EF90DF90CF900895DF92EF922A
:105B7000FF920F931F93CF93DF93D82E862FBA01F6
:105B8000213041F4675F7F4F9B0140E050E0695056
:105B900070400EC0223029F020E030E040E050E0BC
:105BA00007C0625070409B0140E050E06E5F7F4F45
:105BB000E82EFF2482ED92E0E80EF91E8B01E7014A
:105BC0000FC0F881E0E0898190E08E2B9F2BA0E050
:105BD000B0E0280F391F4A1F5B1F22960250104069
:105BE0000230110570F7CB018E7FD701A80FB91FC6
:105BF0006817790779F08C9190E0A0E0B0E0BA2FB7
:105C0000A92F982F882702C040E050E0280F391FA5
:105C10004A1F5B1FCA01AA27BB270097A105B10530
:105C200099F7C90180959095ED2DF0E0EE52FD4F6A
:105C300090838183DF91CF911F910F91FF90EF901F
:105C4000DF9008951092EA021092EB0280E48093B4
:105C5000E6021092E7028093E80288E16EE044E1F8
:105C600050E020E00E94B62D0895282F662321F0F1
:105C70008091F7028617E1F48091F8028823C1F43D
:105C80008091F9028833A1F48091F5028B3781F479
:105C9000E22FF92F8091240383838091250382834F
:105CA00080912603818380912703808381E008957A
:105CB00080E008950F931F93BC0102ED12E0C8012C
:105CC0000E946534C801069668EF7AE00E94653448
:105CD0001F910F910895EF92FF920F931F937B01F5
:105CE0000E945A2E00EF12E0C801B7010E946D34E5
:105CF000C80104976EEF7AE00E946D341F910F91F6
:105D0000FF90EF900895EF92FF920F931F93CF9320
:105D1000DF937C01EB018A0183E29BE00E946B2E02
:105D20008881807F803E49F088819981AA81BB81EA
:105D30008F5F9F4FAF4FBF4F31F482ED92E06DE721
:105D400072E00E94653488E08093DE021092DF02E8
:105D500080EE92E069E878E049E050E00E94500669
:105D60001092E20281E18093E9021093F60200931F
:105D7000F702F092F402E092F5021092F80210920B
:105D8000FA021092FB02DF91CF911F910F91FF90C9
:105D9000EF900895EF92FF920F931F9308ED12E09A
:105DA000C8010E945A2E74E1E72EF12CE00EF11E7C
:105DB000C8014896B7010E946D34C7016EEF7AE0C2
:105DC0000E946D340E94222E1F910F91FF90EF9040
:105DD0000895BC0181E08093180B86E09BE00E944F
:105DE0006D3408950F931F938C0188969093E2026F
:105DF0008093E3020E94222E109204031092050366
:105E0000045E1F4F82E36AE1A80122E00E94B62DE2
:105E1000C8014A960E94C5381F910F910895EF92CC
:105E2000FF920F931F937C0180912B0B90912C0B71
:105E3000A0912D0BB0912E0B2B2F332744275527E4
:105E40002093F802A093F9029093FA028093FB0248
:105E500060930103C7010E94F22E00E010E08091E0
:105E60002B0B90912C0BA0912D0BB0912E0B8E0D26
:105E70009F1DA01FB11F80932B0B90932C0BA09301
:105E80002D0BB0932E0B1F910F91FF90EF90089563
:105E9000CF93DF939C01862F806180930103643050
:105EA00029F02115310511F421E030E09091F6023E
:105EB0008091F4028093F6029093F4029091F7029D
:105EC0008091F5028093F7029093F502CBEFD2E038
:105ED0008881A901480F511D2C814C832883252FCF
:105EE0003327219752E0C73FD50791F71D861E86BD
:105EF00080E589871092E20288E28093E3020E94A3
:105F0000CA2E84E08B871C8682E36AE14CE150E074
:105F100022E00E94B62D86E390E00E94C538DF9112
:105F2000CF9108958091290B90912A0B60E00E94F7
:105F3000482F8091F80290E0A0E0B0E0BA2FA92F9E
:105F4000982F88272091F902820F911DA11DB11D64
:105F5000BA2FA92F982F88272091FA02820F911D1E
:105F6000A11DB11DBA2FA92F982F88272091FB02C0
:105F7000820F911DA11DB11D80932B0B90932C0BB3
:105F8000A0932D0BB0932E0B08950F931F938C01AC
:105F90008091290B90912A0B60E00E94482F89E1A3
:105FA00080930103C8010E94F22E1F910F91089562
:105FB000E82FA091E202B091E302F091000340913A
:105FC000F60250E0292F30E04217530709F08EC047
:105FD0008091F7028E1709F089C080910103E82FA4
:105FE00081FF4EC01092E2028CE28093E3020E9495
:105FF000CA2E82E1809301039091F6028091F4020F
:106000008093F6029093F4029091F7028091F5024A
:106010008093F7029093F502EBEFF2E021E030E09D
:106020008081A901480F511D44831082252F3327F9
:10603000319752E0E73FF50799F7158616861182EA
:1060400012828091AA01838314828D5F8093AA01BA
:1060500082E0818B84E0828B95E0938B148A80E6CA
:106060008187938788E7848782E36AE140E250E092
:1060700022E00E94B62D8AE390E00E94C53836C027
:1060800084FF34C04F2F50E084E0559547958A95A2
:10609000E1F79A2F80E02B2F30E0282B392BCA0113
:1060A000880F991F880F991F281B390B24513040E6
:1060B00037FF02C020E030E030932A0B2093290BF9
:1060C000232B69F09A01220F331F220F331F2E5DFD
:1060D0003F4F685070406217730740F009C0E0FFFF
:1060E00005C080E090E060E00E94482F20E030E0B2
:1060F000C90108950F931F93DF93CF930F92CDB7EC
:10610000DEB78C01045E1F4F1093E2020C51104069
:10611000802F845E8093E30289830E94222E085F91
:106120001F4F1093F802898184518093F902085F10
:106130001F4F88E26AE1A80121E00E94B62DC80144
:106140004A960E94C5380F90CF91DF911F910F9111
:106150000895FF920F931F939C01F62E83E29BE01C
:10616000B9010E946B2E0EED12E088E08093DE02F2
:106170001092DF02C801029669E878E049E050E039
:106180000E9450068CE48093E30281E18093E9024F
:106190000E94222E1092F6028BE78093F7028AE08B
:1061A0008093F402F092F5021092F80288E3809353
:1061B000F9021092FA021092FB02025E1F4F80E376
:1061C000F80111928A95E9F7C80160E479E04AE0A4
:1061D00050E00E94500688E26AE140E450E021E08D
:1061E0000E94B62D8AE590E00E94C5381F910F915C
:1061F000FF900895EF92FF920F931F93BC0183E2EB
:106200009BE00E946B2E0EED12E038E0F32EF09230
:10621000DE021092DF02C801029669E878E049E0E8
:1062200050E00E94500684E58093E302EE24E3945C
:10623000E092E9020E94222EF092F4021092F502FE
:106240001092F6021092F70285E08093F802809196
:10625000010B8093F9021092FA02E092FB02C8014E
:106260004E9662E470E048E350E00E94660684E2E5
:1062700062E240E450E020E00E94B62D82E690E029
:106280000E94C5381F910F91FF90EF900895DF9203
:10629000EF92FF920F931F93CF93DF93EC018091C6
:1062A000160B882319F0CE010E948528209709F04B
:1062B000BFC08091180B8570F1F18091A70190917A
:1062C000A801892BC1F50E94FD378823A1F18DE734
:1062D00092E00E945A2E88E08093DE02A6E0FA2E19
:1062E000F092DF0280EE92E061E878E048E050E072
:1062F0000E94500602EF12E0D8011D92FA94E9F7CD
:10630000C8010A9768EF7AE00E946534C8010696D2
:1063100066E07BE00E946D34C80104976EEF7AE07E
:106320000E946D348091180B88608093180B8AE26C
:1063300090E00E94C5388091A7019091A801019634
:106340009093A8018093A7018091190B813009F0E7
:1063500002C28091180B81FFFEC102E00093190B6D
:106360008091A9018F5F8093A9018F7110911A0B01
:106370001295110F107E182BE0901B0BD0901C0B68
:1063800083E29BE062E17BE00E946B2EF8E0FF2E4F
:10639000F092DE021092DF0280EE92E069E878E08F
:1063A00049E050E00E9450068CE28093E30286E0D0
:1063B0008093E9020E94222EE092F602D092F70228
:1063C0008BE08093F4021093F502E8EFF2E0DF0136
:1063D0001D92FA94E9F78091AA018093FA028D5FE9
:1063E0008093AA0180E6809300030093010383E079
:1063F000809302031092030310920403109205038A
:1064000010920603109207030093080384E0809320
:10641000090300930A0386E280930B0382E36AE197
:1064200040E250E022E00E94B62D8AE390E0AEC048
:106430008091F0028F3E79F48091F1028F3F59F400
:106440008091F2028F3F39F48091F3028A3F19F470
:106450002AE230E082C1C932D10508F47CC1109132
:10646000DE02183009F082C18091DF02863009F027
:106470007DC188EF92E06EEF7AE044E050E00E9448
:106480005906009709F072C18091E702813029F521
:1064900088ED92E00E945A2E1092E60282E08093EC
:1064A000E70282EF92E068EE72E00E94653488EEC7
:1064B00092E068EF7AE00E94653488EF92E06EEE39
:1064C00072E00E946D348EEE92E06EEF7AE00E94F0
:1064D0006D348AE290E00E94C5388091180B83FFEA
:1064E0003AC11091E702123009F035C18EEE92E008
:1064F00066E07BE044E050E00E945906009709F016
:106500002AC183E29BE068EE72E00E94653410933A
:10651000180B21C1183009F01EC18091DF028823B9
:1065200009F019C18091E002853409F014C180EFAF
:1065300092E06EEF7AE044E050E00E945906009746
:1065400009F009C18091E902813019F58091F402C6
:106550008830F9F4E0911D0BF0911E0B309719F083
:106560008CEE92E009950E94CA2E1092F40280915E
:10657000F602883F28F08091F7028F5F8093F70240
:106580008091F602885F8093F602CE010E94C538A2
:10659000E2C00E940D3B882351F08091E9028131D5
:1065A00031F4CE010E94123B882309F0D4C0C633D7
:1065B000D10528F48091E902863009F0CCC08091A1
:1065C000F6028B3009F0BEC08CEE92E062E17BE017
:1065D00044E050E00E945906009709F0BCC0809149
:1065E0000103382F82FF13C0E0911F0BF091200BA5
:1065F000309759F08091F70282958695877063E015
:1066000040E050E020E030E0099585E090C09091B6
:10661000E20280E02091E302022F10E0082B192B08
:1066200080910003482F50E0E4E055954795EA95A6
:10663000E1F7CA01880F991F880F991F081B190BD2
:106640000451104017FF02C000E010E08091190BC8
:10665000823079F531FF21C034FF1FC080E090E027
:1066600060E00E94482F88E180930103E091210BB4
:10667000F091220B309719F420E030E007C08091B0
:10668000F50282958695877009959C0183E0809339
:10669000190BC9010E94F22E5EC081E08093190B94
:1066A00034FF03C080E090E002C0C801019664E0BE
:1066B00046C0833081F50115110579F1E0911F0B7A
:1066C000F091200B309749F1440F551F440F551F8F
:1066D000CE0108974E5D5F4F8417950708F4AC0113
:1066E000C801840F951FC817D90710F0980103C07F
:1066F0009E01241B350B8091F70282958695877049
:1067000060E009958091170B882319F0C80168E0B3
:1067100016C0C80108C08530F1F030FF0BC08330CF
:10672000D1F0C801019669E00E94482F86E080936D
:10673000190B11C00115110571F0C80160E00E942C
:10674000482F09C08091A5019091A601BE010E9429
:10675000D82F9C0102C020E030E0C901DF91CF9129
:106760001F910F91FF90EF90DF900895CA32D105ED
:1067700008F0D0CEF0CFBC018091E9028130A1F4C5
:106780008091F402882381F48091FC02823461F4C8
:106790008CEE92E044E050E00E9459069C0180E0BB
:1067A000232B19F481E0089580E00895CF93DF93BF
:1067B000DC01EB01722F632F822F932F9C01F901D3
:1067C00050E016C08081981771F43196808188233B
:1067D00071F411968C918D3331F4872F962F9C0193
:1067E000F90151E004C0872F962F9C01F901119601
:1067F0009C91992339F0903229F09A3019F0552361
:1068000009F304C0513011F030E018C06A2F50E095
:106810004150504002C0299311963A2F361B2C91BB
:10682000222359F0203249F02A3039F0263229F05B
:10683000832F90E08417950774F31882832FDF91DC
:10684000CF910895CF93DF93FC01EC0137C08B32D9
:1068500011F480E231C0853279F5DF011196918122
:10686000392F30533A3070F0892F8156863010F42A
:10687000375208C0892F8154863010F030E002C0B2
:10688000392F3753FD01319611962C91922F905349
:106890009A3070F0822F8156863010F4975208C0DB
:1068A000822F8154863010F090E002C0922F9753CF
:1068B000832F8295807F892B8993319680818823CD
:1068C00031F61882DF91CF910895DC01FB0186E05B
:1068D00001900D928150E1F708959C01FB018081A8
:1068E0009181A281B381F90180839183A283B383D3
:1068F00008958F929F92AF92BF92CF92DF92EF92C4
:10690000FF920F931F93CF93DF937B018C01EA01DA
:106910002CE330E040E050E00E94404F6883C80123
:10692000B7012CE330E040E050E00E94404F122FCE
:10693000032FF42EE52E622F732F842F952F2CE337
:1069400030E040E050E00E94404F6983612F702F9B
:106950008F2D9E2D2CE330E040E050E00E94404F10
:10696000122F032FF42EE52E622F732F842F952FD5
:1069700028E130E040E050E00E94404F6A83612F00
:10698000702F8F2D9E2D28E130E040E050E00E94D6
:10699000404F79018A01C801B7016C5F7F4F8F4F6B
:1069A0009F4F27E030E040E050E00E94404F6F5F93
:1069B0006B8320E0AA24BB24650101C02F5F822ED7
:1069C0009924F401EE54F84FCF0183709070892B15
:1069D00099F4CF0164E670E00E942D4F892B39F4C1
:1069E000CF0160E971E00E942D4F892B29F48EE6DA
:1069F00091E0A0E0B0E004C08DE691E0A0E0B0E05E
:106A0000A80EB91ECA1EDB1EC501A0E0B0E0E81644
:106A1000F9060A071B0790F62E83F401EE54F84F8F
:106A200083E0882E912C8E229F228114910499F468
:106A3000CF0164E670E00E942D4F892B39F4CF011D
:106A400060E971E00E942D4F892B29F48EE691E0D8
:106A5000A0E0B0E004C08DE691E0A0E0B0E0A81AAC
:106A6000B90ACA0ADB0A980187010A191B092C090D
:106A70003D09CF0164E670E00E942D4F7C01CF01FB
:106A800060E971E00E942D4FAC01E3E8F2E060E0C4
:106A9000613051F48114910449F4E114F10441F49A
:106AA0004115510529F002C0808103C08CE101C06D
:106AB0008DE190E0A0E0B0E0081719072A073B0736
:106AC00040F0081B190B2A0B3B0B6F5F31966C30A3
:106AD000F9F66F5F6D83802F8F5F8C83DF91CF918D
:106AE0001F910F91FF90EF90DF90CF90BF90AF90EC
:106AF0009F908F900895EF92FF920F931F937B01C9
:106B00008C018091460B9091470BA091480BB0915E
:106B1000490BE816F9060A071B0771F0C801B7010F
:106B20004BE35BE00E947934E092460BF092470B16
:106B30000093480B1093490B1F910F91FF90EF901A
:106B400008950E947B352091410B30E02E54384F40
:106B5000C90108950E947B358091400B90E0089513
:106B60000E947B3580913E0B90E008950E947B351A
:106B700080913F0B90E008950E947B3580913C0B03
:106B800090E008950E947B3580913D0B90E0089540
:106B90004F925F926F927F928F929F92AF92BF922D
:106BA000CF92DF92EF92FF920F931F93CF93DF93D9
:106BB0004C01DC0116961C91612F70E080E090E0A2
:106BC00020E833E341EE51E00E94EE4E5B016C01A0
:106BD00022EB37E0E12FF0E0EE54F84F1DC0C90181
:106BE00083709070892BB1F4C90164E670E00E9453
:106BF0002D4F892B39F4C90160E971E00E942D4FB6
:106C0000892B41F480E891E5A1E0B0E0A80EB91E1F
:106C1000CA1EDB1E2F5F3F4F2E173F0701F7D4011F
:106C200015968C91482E5524C90164E670E00E94A7
:106C30002D4F7C01C90160E971E00E942D4F8C014C
:106C4000C1E0D0E093E0692E712C6222732227C04C
:106C5000C230D10591F46114710479F4E114F104A6
:106C600019F40115110549F480E89BE3A6E2B0E0B0
:106C7000A80EB91ECA1EDB1E11C0FE01EE57FD4F45
:106C8000608170E080E090E020E831E541E050E094
:106C90000E94EE4EA60EB71EC81ED91E2196C41520
:106CA000D505B4F2D40112966C9170E080E090E0CA
:106CB00020E13EE040E050E00E94EE4E7B018C017E
:106CC000F401618170E080E090E02CE330E040E08E
:106CD00050E00E94EE4EE60EF71E081F191FD40169
:106CE0008C91E80EF11C011D111D14966C9170E041
:106CF00061507040882777FD8095982F20E831E516
:106D000041E050E00E94EE4EE60EF71E081F191FEC
:106D1000EA0CFB1C0C1D1D1DB701C801DF91CF91B2
:106D20001F910F91FF90EF90DF90CF90BF90AF90A9
:106D30009F908F907F906F905F904F900895609399
:106D4000AB017093AC018093AD019093AE010895B7
:106D50006093310B7093320B8093330B9093340B11
:106D60002091AB013091AC014091AD015091AE0149
:106D7000260F371F481F591F2093350B3093360BB2
:106D80004093370B5093380B82E090E090933A0B8E
:106D90008093390B0E94CD4A6093420B7093430B52
:106DA0008093440B9093450B0895EF92FF920F93BD
:106DB0001F931CC02F5F3F4F4F4F5F4F2093310BEE
:106DC0003093320B4093330B5093340B88EE93E0A7
:106DD000A0E0B0E0E80EF91E0A1F1B1FE092420B74
:106DE000F092430B0093440B1093450B0E94CD4A45
:106DF000E090420BF090430B0091440B1091450B37
:106E00006E197F09800B910B2091310B3091320B61
:106E10004091330B5091340B685E7340804090403A
:106E200048F68091350B9091360BA091370BB091BD
:106E3000380B281739074A075B07E8F0E0912F0B5A
:106E4000F091300B3097B9F0099561157105810506
:106E5000910519F00E94A8360EC020E030E0809124
:106E6000390B90913A0B892B11F021E030E03093EF
:106E70003A0B2093390B6091310B7091320B80915A
:106E8000330B9091340B1F910F91FF90EF90089569
:106E90009093300B80932F0B8091310B9091320B9C
:106EA000A091330BB091340B8093350B9093360B3C
:106EB000A093370BB093380B0E94D53608950E94EB
:106EC000D5360E947B3580913E0B90E008958091ED
:106ED0004C0B61E00E94724978940895FF920F93E1
:106EE0001F93082F162FF42EF89480914C0B60E01E
:106EF0000E9472491F71102B1EBD0DB407FEFDCFFD
:106F0000FEBC0DB407FEFDCF0E9467371F910F91A5
:106F1000FF9008951F93182F282F30E020763070AF
:106F200080914D0B90E02817390799F080EA6FE1C6
:106F300043E00E946E37412F407640934D0B50E066
:106F400085E0559547958A95E1F780E86FE10E94C5
:106F50006E371F9108950F931F93182F062F0E94CD
:106F60008A3780E4612F402F0E946E371F910F9166
:106F700008950F931F93182F072F0E94AB37812F6F
:106F80008F5F602F0E94AB371F910F91089588E3A8
:106F900060EB0E94AB37089588E361EB0E94AB374A
:106FA00008950F931F93182F062FF89480914C0B80
:106FB00060E00E947249802F8F71812B8EBD0DB4CD
:106FC00007FEFDCF1EBC0DB407FEFDCF07FF04C0BA
:106FD0001EBC0DB407FEFDCF1EB50E946737812F82
:106FE0001F910F9108951F93182F0E948A3780E0F8
:106FF000612F0E94D1371F91089584ED61E10E94B5
:10700000AB3782ED61E00E94AB378AEE0E94F33726
:1070100080FDFBCF82ED60E00E94AB3789ED0E94DE
:10702000F33790E0969587959695879581700895AA
:107030000F931F93CF93DF93EC018B01F894809112
:107040004C0B60E00E9472498AE38EBD0DB407FECE
:10705000FDCF09C01EBC0DB407FEFDCF8EB5F801F3
:1070600081938F0121972097A9F70E946737DF91BD
:10707000CF911F910F9108950F931F93DF93CF939B
:1070800000D000D000D0CDB7DEB789E30E94F3373F
:10709000882319F400E010E048C060914E0B709115
:1070A0004F0B80E00E94B93786E090E0BE016F5F31
:1070B0007F4F0E94183889819A8190934F0B80935B
:1070C0004E0B2B813C81E0914A0BF0914B0B8D8153
:1070D00087FD03C000E010E00EC0245030408F0157
:1070E000015010402017310708F48901C80162EDF2
:1070F00072E00E941838F801EE52FD4F1082609144
:107100004E0B70914F0B8CE06130780724F08CE0CF
:107110006FEF7BE003C0615070408CE00E94B93794
:1071200080E86EE140E40E946E37C80126960FB6F3
:10713000F894DEBF0FBECDBFCF91DF911F910F91AD
:1071400008950F931F93CF93DF938C01EB01F89475
:1071500080914C0B60E00E9472498AE78EBD0DB4AD
:1071600007FEFDCF08C088818EBD0DB407FEFDCFA0
:1071700021960150104001151105A9F70E946737AB
:10718000DF91CF911F910F910895CF93DF93EC0181
:107190000FC08CE10E94F33781FF0AC080E86FE1E5
:1071A00040E80E946E3780EA6FE140E80E946E3747
:1071B00080E06FE10E94D13783FDEBCF82E060E099
:1071C0007CE00E94B937BE016050744F86E00E9497
:1071D000B9378AE760E040E00E946E37CE0162ED89
:1071E00072E00E94A13880E86FE148E00E946E37AB
:1071F000DF91CF91089584E061E00E94334984E0FB
:1072000061E00E94724985E061E00E94334987E0B5
:1072100061E00E94334986E060E00E94334985E0E6
:1072200061E00E94724985E060E00E94724987E057
:1072300060E00E94724980E58CBD8DB581608DBD96
:1072400008951F93CF93DF93EB01142F90934B0B73
:1072500080934A0B0CB406FC02C00E94FB381093CA
:107260004C0B812F61E00E9433490E9467378FEFFA
:1072700060E04FEF0E946E3762E070E080E090E0E7
:107280000E94DB4A80E06DE10E94D1378823D1F370
:1072900010924F0B10924E0B88E060E070E00E945D
:1072A000B9378CE060E070E00E94B9378AE06FEF98
:1072B0007BE00E94B93784E060E07CE00E94B9374F
:1072C00086E06FEF71E10E94B9370E94CC3788E207
:1072D0006FE370E30E94B93780E369EF77EF0E94B4
:1072E000B93780EC6DE00E94AB3781EC60E00E9422
:1072F000AB3780E862EC42E30E946E3786EC62E1D5
:107300007CE00E94B93784EC62E10E94AB378AECE2
:107310006CED75E00E94B93784EE68810E94AB374E
:1073200085EE69810E94AB3782EE6A810E94AB379D
:1073300083EE6B810E94AB3780EE6C810E94AB378D
:1073400081EE6D810E94AB3784ED60E10E94AB3726
:1073500086ED60E071E00E94B9378AEE0E94F33753
:1073600080FDFBCF8FE10E948A3780E86BE140EC23
:107370000E946E3780E86FE144E00E946E3782E73A
:107380000E94F337863008F08F5FDF91CF911F9115
:107390000895482F6AE00E940D4F282F30E084E0C6
:1073A000220F331F8A95E1F7842F0E940D4F892FFA
:1073B000820F0895EF92FF920F931F937C010BEEC3
:1073C0001BE0C80168E670E00E94BC43C80160E0B1
:1073D0000E943E44F70180810E94C939682FC8018C
:1073E0000E943E44F70181810E94C939682FC8017B
:1073F0000E943E44F70182810E94C939682FC8016A
:107400000E943E44F70183810E94C939682FC80158
:107410000E943E44F70184810E94C939682FC80147
:107420000E943E44F70185810E94C939682FC80136
:107430000E943E44F70186818E510E94C939682F0F
:10744000C8010E943E44C8010E9481441F910F91CF
:10745000FF90EF9008950F931F930BEE1BE0C80170
:1074600068E670E00E94BC43C80160E00E943E44B0
:10747000C8010E9481441F910F910895DF92EF92FD
:10748000FF920F931F937C010BEE1BE0C80168E68F
:1074900070E00E94BC43C80160E00E943E44C80105
:1074A0000E948144C80168E670E047E050E00E9415
:1074B0009244C8010E94CF43282F2F7722952F7026
:1074C0009AE0D92E2D9D900111248F70820FF70123
:1074D0008083C8010E94CF43282F22952F702D9DB5
:1074E000900111248F70820FF7018183C8010E94DF
:1074F000CF43282F2F7322952F702D9D900111249B
:107500008F70820FF7018283C8010E94CF43282F1A
:1075100022952F702D9D900111248F70820FF701FD
:107520008383C8010E94CF43282F22952F702D9D61
:10753000900111248F70820FF7018483C8010E948B
:10754000CF43282F22952F702D9D900111248F70ED
:10755000820FF7018583C8010E94CF43282F2F7027
:10756000225E82958F708D9DC0011124280FF70136
:1075700026831F910F91FF90EF90DF9008950F9356
:107580001F93DF93CF93CDB7DEB727970FB6F8944D
:10759000DEBF0FBECDBF8E010F5F1F4FA8010E943F
:1075A0007934898180688983C8010E94DA398981A8
:1075B0008F778983C8010E94DA3927960FB6F8942D
:1075C000DEBF0FBECDBFCF91DF911F910F91089508
:1075D0000F931F93DF93CF93CDB7DEB727970FB6E7
:1075E000F894DEBF0FBECDBF8E010F5F1F4FC801E5
:1075F0000E943E3AC8010E94C83527960FB6F894FB
:10760000DEBF0FBECDBFCF91DF911F910F910895C7
:107610008BEE9BE00E94964408958091780B811137
:1076200081E00895CF92DF92EF92FF920F931F9324
:10763000CF93DF93C0E5DBE0CC24DD2430E029C02C
:107640002A814B818091F60290E0042F10E0801790
:107650009107D9F49091F7029217B9F48C8188239D
:10766000A1F02091F90230E028503040F090F8026B
:10767000EE242E0D3F1DE881F981892F942F6CEEA9
:1076800072E04CEF52E0099531E00894C11CD11C26
:1076900025968091780B90E0C816D9068CF2832F3E
:1076A000DF91CF911F910F91FF90EF90DF90CF90DE
:1076B0000895E091A20BF091A30B09950895DB01C9
:1076C000482F50E0495F5F4F84E0440F551F8A9573
:1076D000E1F750961C92509720E030E0F999FECFE8
:1076E000C901840F951F92BD81BDF89A80B5FD0137
:1076F000E20FF31F8083882331F02F30310519F01A
:107700002F5F3F4FEBCF0895DB01482F50E0495FDB
:107710005F4F94E0440F551F9A95E1F750961C92E5
:10772000509720E030E0FD01E20FF31FE081F9996E
:10773000FECF1FBAC901840F951F92BD81BDE0BD68
:107740000FB6F894FA9AF99A0FBEEE2331F02F3063
:10775000310519F02F5F3F4FE6CF089580ED93E09C
:10776000FC01E853F84FE081F999FECF1FBA92BDB2
:1077700081BDE0BD0FB6F894FA9AF99A0FBE019652
:1077800023E0863D920761F70895282F277086959C
:107790008695869590E0662369F0FC01EE56F44FDD
:1077A00081E090E002C0880F991F2A95E2F72081BE
:1077B000282B0DC0FC01EE56F44F81E090E002C092
:1077C000880F991F2A95E2F780952081282320832E
:1077D00008951092920B1092930B1092940B1092AA
:1077E000950B1092960B1092970B0895EFEAF1E02B
:1077F00020E030E0F999FECF32BD21BDF89A80B586
:1078000080832F5F3F4F35962232310599F7809163
:10781000FA018F5F8093900B90E023E0880F991F0F
:107820002A95E1F78093910B0895E4E5F2E081E277
:1078300090E02081F999FECF1FBA92BD81BD20BD95
:107840000FB6F894FA9AF99A0FBE019735972FEF71
:107850008F3F920771F78091FA018F5F8093900BB1
:1078600090E033E0880F991F3A95E1F78093910BF0
:107870000895AC01FB010FC0F999FECF1FBADA01E0
:10788000A80FB11DB2BDA1BD20BD0FB6F894FA9AE4
:10789000F99A0FBE31968E2F861B2081222361F725
:1078A000F999FECF1FBA480F511D52BD41BD10BC02
:1078B0000FB6F894FA9AF99A0FBE0895AC01FB013D
:1078C0008E2F861BF999FECF9A01280F311D32BDEC
:1078D00021BDF89A80B58083882311F03196F0CFCE
:1078E0000895582F282F392FF9018E2F851BF999CC
:1078F000FECF90E0805C9F4F92BD81BDF89A80B52D
:107900009081882331F0992349F0891739F4319611
:10791000ECCF80E0992319F481E0089580E0089588
:10792000CF92EF920F9389E79BE063E142E124E17C
:1079300005E176E1E72E57E1C52E0E94FA480F9146
:10794000EF90CF900895EF92FF920F931F93CF93F4
:10795000DF93E82E162F042FF22E662321F06230DB
:1079600081F4222371F08E2D0E94C649892B11F0DB
:1079700000E024C0FF2011F480E001C080E8082B63
:107980001DC0C0E0D0E08E2D0E94C649892B81F435
:10799000113031F0123061F483E0C032D80744F482
:1079A00061E070E080E090E00E94DB4A2196EBCF3E
:1079B000FF2019F4C052D3400CF00068802FDF91F3
:1079C000CF911F910F91FF90EF9008950F931F9308
:1079D000082F1091A40B107861E070E080E090E037
:1079E0000E94DB4A8FE10E94C649892B21F48FE176
:1079F000602F41E013C08EE10E94C649892B21F41B
:107A00008EE1602F42E00AC08DE10E94C649892BB9
:107A100011F040E007C08DE1602F44E0212F0E946B
:107A2000A33C482F8091A40B90E08F709070242F7E
:107A300030E0892B39F42F703070232B71F0842FB4
:107A4000806406C02F703070232B39F4842F80623D
:107A50004093A40B1F910F910895842FF9CF8BE0D1
:107A60000E94C64940E020911D0230E08217930732
:107A700009F041E0440F440F80918E0B8B7F842BE3
:107A800080938E0B0895EF92FF920F931F938C01BA
:107A9000E9E7EE2EEBE0FE2E6AE070E00E942D4F4B
:107AA000C7014AE050E00E94724CC8016AE070E0F1
:107AB0000E942D4FBC01C7014AE050E00E94724C69
:107AC0001F910F91FF90EF900895CF93DF93EC01FA
:107AD00004C089E79BE00E94B24BFE0121966491AD
:107AE0006623B9F7DF91CF9108950F931F93CF933A
:107AF000DF938C01462F89E79BE060E00E940D48F0
:107B0000E80104C089E79BE00E94B24B9E01201B64
:107B1000822FFE01219664916623A1F7992787FDA4
:107B20009095C0E1D0E0C81BD90B05C083E39BE072
:107B30000E94653D2197D7FFF9CFDF91CF911F912B
:107B40000F910895EF92FF920F931F93CF93DF93BE
:107B50007C018C01000F111F000F111F0E0D1F1D46
:107B600001551E4FF8018281938160E00E94753DAE
:107B700080E09BE061E00E94753D89E79BE060E06A
:107B800041E00E940D48F801848180FF05C089E72B
:107B90009BE00E94F14704C089E79BE00E94FB47FD
:107BA000F3E1EF16F10409F45EC084E1E816F10494
:107BB00054F4E1E0EE16F104B1F0FCE0EF16F1044C
:107BC00009F08CC065C08BE1E816F10409F46AC0C5
:107BD000ECE1EE16F10409F475C0F4E1EF16F104DE
:107BE00009F07CC047C08091B401C82FD0E0E09775
:107BF000D7FD05C08EEF9AE00E94653D07C08CEF6F
:107C00009AE00E94653DD095C195DF4FCE0164E0BA
:107C100070E00E942D4F89E79BE04AE050E00E940F
:107C2000724C8AEF9AE00E94653DCE0164E070E0FC
:107C30000E942D4FBC01B4E0660F771FBA95E1F7A3
:107C4000681B790B29F487EF9AE00E94653D06C016
:107C500089E79BE04AE050E00E94724C82EF9AE094
:107C60000E94653D60C080EF9AE00E94653D609192
:107C70000E0220C0809113028C3320F08EEE9AE029
:107C80000E94653D6091130270E06C53704007C024
:107C90007091F00160E08091EB01680F711D89E740
:107CA0009BE00BC0609136028DE070E00E94194AA3
:107CB0006091360289E79BE070E04AE050E00E9464
:107CC000724C31C080913B026FEF70E0681B71090C
:107CD0008CE00E94194A60913B02ECCFF701EE0F55
:107CE000FF1FEE0FFF1FEE0DFF1DE155FE4F8181BF
:107CF0006081813051F4662319F487EE9AE002C066
:107D00008AEE9AE00E94653D07C089E79BE070E03B
:107D10004AE050E00E94724C87E1E816F10419F441
:107D200085EE9AE011C0C7014397029720F0E8E181
:107D3000EE16F10419F480EE9AE006C0F1E1EF16B8
:107D4000F10421F48BED9AE00E94653DDF91CF9123
:107D50001F910F91FF90EF900895EF92FF920F9374
:107D60001F93182F092F0E94A23D212F302FC901E8
:107D70008C013AEAE32E82E00E94E63C482F282F4D
:107D800030E0C9018F70907082309105D1F084305D
:107D9000910551F1019709F066C0F801EE0FFF1F40
:107DA000EE0FFF1FE00FF11FE155FE4F848180FFB2
:107DB0005DC090818181891709F458C09F5F9083CD
:107DC00055C0F801EE0FFF1FEE0FFF1FE00FF11F70
:107DD000E155FE4F848180FF46C08081882309F4ED
:107DE00042C0815080833FC046FF3DC047FF0BC06B
:107DF00080915402882311F0E09254020E94153CB5
:107E0000FF24F39434C00330110541F48091BE0186
:107E1000882309F1FF240CE010E029C00C30110583
:107E200021F4FF240EE010E022C00531110541F4D9
:107E300080911802882379F4FF2407E110E017C02D
:107E40000231110541F480910902882321F4FF24B5
:107E500005E110E00CC0C801019662E270E00E94EA
:107E60002D4F8C0103C0442309F485CFFF24C801A2
:107E70000E94A23DFF2009F47ECF89E79BE00E948B
:107E8000FB471F910F91FF90EF9008950F931F9361
:107E9000CF93DF93482F062F89E79BE060E00E9495
:107EA0000D4880918F0B8F7019F482E29BE010C017
:107EB00080E29BE00E94653D60918F0B6F7089E7C7
:107EC0009BE070E04AE050E00E94724C8EE19BE043
:107ED0000E94653D80918E0B80FD03C082E19BE096
:107EE0000AC081FD06C082FF0AC080911802882363
:107EF00031F086E09BE061E00E94753D26C0E09194
:107F00008F0BEF70F0E0EE56F44F1081C1E0D0E03F
:107F100080918F0B8F7051F48091090290E0C81707
:107F2000D90721F410FD06C06DE405C010FD02C0A4
:107F30006FE501C0602F89E79BE00E94B24B21965C
:107F4000C930D10511F01695E3CF81E09BE00E9486
:107F5000653D89E79BE06EE041E00E940D4860E0EE
:107F600080918F0B82958F7009F061E089E79BE02B
:107F70000E94BF4789E79BE06FE041E00E940D4807
:107F800080918E0B86FF05C089E79BE062E00E942E
:107F9000BF47DF91CF911F910F910895EF92FF920C
:107FA0000F931F93CF93DF938C017B0189E79BE0B5
:107FB0000E943C4889E79BE060E040E00E940D4859
:107FC000C0E0D0E0F801EC0FFD1F608189E79BE085
:107FD00070E04AE050E00E94724C88E29BE00E9410
:107FE000653D2196C330D10569F7F801638189E7C2
:107FF0009BE070E04AE050E00E94724C89E79BE011
:1080000060E041E00E940D4886E29BE00E94653DF1
:1080100089E79BE0B7014AE050E00E94724CDF9193
:10802000CF911F910F91FF90EF900895EF92FF92E3
:108030000F931F93CF93DF9383E060E00E94724918
:1080400007E91BE090918E0B90FF0BC091FD09C0DA
:1080500080911802882311F092FD03C0F80160811D
:1080600001C060E0C7E0D0E0E62EFF2486E160E0DA
:108070000E947249B7010C2E02C0759567950A944B
:10808000E2F7617085E10E94724986E161E00E9439
:1080900072492197FFEFCF3FDF0741F701501040B2
:1080A0008BE00139180771F683E061E00E947249A4
:1080B000DF91CF911F910F91FF90EF9008958091E4
:1080C0008E0B8D7F80938E0B0E9416400895DF9259
:1080D000EF92FF920F931F93D82E882309F10E94ED
:1080E000D5367B018C016D2D70E080E090E020E1C1
:1080F0003EE040E050E00E94EE4EE60EF71E081F04
:10810000191FE0929E0BF0929F0B0093A00B10930F
:10811000A10B80918E0B826080938E0B0E94164083
:108120001F910F91FF90EF90DF90089580918E0B3B
:108130008E7F80938E0B0E9416400E94153C0895FE
:1081400080918E0B816080938E0B0E9416400E945E
:10815000153C0895AF92BF92CF92DF92FF920F939A
:108160001F93CF93DF935B016C01FF24C1E0D0E04C
:108170003CC089E79BE00E943C4889E79BE060E0C7
:1081800040E00E940D480F2D10E0B8016F5F7F4F57
:1081900089E79BE04AE050E00E94724C1092920BFB
:1081A0001092930B1092940B1092950B1092960BC9
:1081B0001092970B43E0169507954A95E1F70E56F6
:1081C000144F8F2D87709E0102C0220F331F8A9596
:1081D000E2F7C901F8012081282B20830E94164074
:1081E000C601B5010E94DB4AF3948091910BF81609
:1081F00008F4BFCFFF24FBCF64EF71E080E090E094
:108200000E94DB4AF999FECF12BC11BCF89A90B5D6
:10821000943620F48AE0989F902D1124993C59F4CB
:10822000F999FECF81E290E092BD81BDF89A80B5C8
:108230008A3A09F089C00E94153C80E490E064E32A
:1082400071E00E94393C80E590E06DE371E00E94AE
:10825000393C85E79BE060E00E94753D86E69BE047
:1082600061E00E94753D80E790E0F999FECF1FBA6A
:1082700092BD81BD10BC0FB6F894FA9AF99A0FBE60
:10828000019628E08030920781F720E730E0E1E0B6
:10829000F0E043E5F999FECF1FBA32BD21BD40BDE4
:1082A0000FB6F894FA9AF99A0FBEF999FECF1FBA51
:1082B0002F5F3F4F32BD21BD21503040CF016AE0DA
:1082C00070E00E942D4F605D60BD0FB6F894FA9A81
:1082D000F99A0FBEF999FECF1FBA2E5F3F4F32BDFC
:1082E00021BDCF016AE070E00E942D4F805D80BD0E
:1082F0000FB6F894FA9AF99A0FBE225F3F4F83E0C7
:108300002037380711F03196C5CF80ED93E02FEF7D
:10831000F999FECF1FBA92BD81BD20BD0FB6F8946A
:10832000FA9AF99A0FBE019633E0863D930781F7DA
:1083300064EF71E080E090E00E94DB4AE091A20BE4
:10834000F091A30B099514C00E94F63B20ED33E099
:10835000F999FECF32BD21BDF89A80B5F901E853F5
:10836000F84F80832F5F3F4F83E0263D380781F72A
:1083700080E00E94E63C90E08F7090708230910522
:1083800021F18430910521F1019709F04CC064E698
:1083900070E080E090E00E94DB4A8DE10E94C649D7
:1083A000892B29F460E273E080E090E00BC06091DB
:1083B000270270E080E090E028EE33E040E050E0FB
:1083C0000E94EE4E0E94AA402EC081E290E020C0A2
:1083D00086E59BE060E00E94753D60ED77E080E01F
:1083E00090E00E94DB4A85E49BE060E00E94753DDE
:1083F00085E39BE061E00E94753D80E00E94E63CE1
:1084000086FFFBCF89E79BE00E943C4880E090E03C
:108410000E94AD3E80915402882329F0E091A20B86
:10842000F091A30B09958CE061E00E9433498DE047
:1084300061E00E943349609136028DE070E00E9455
:10844000194A80913B026FEF70E0681B71098CE064
:108450000E94194A08950E945F3790E0059667E0F0
:1084600070E00E942D4F0895DF92EF92FF920F93DC
:108470001F93D82E0E94D5367B018C0189E79BE0A3
:1084800060E04D2D0E940D48C801B7010E94C23521
:108490000E94433D81E39BE00E94653DC801B70116
:1084A0000E94BC350E94433D8EE29BE00E94653DE8
:1084B0000E942B42E82FF0E0EE0FFF1FE75AFD4F1E
:1084C000808191810E94653D8CE29BE00E94653D28
:1084D000C801B7010E94AA350E94433D8AE29BE091
:1084E0000E94653DC801B7010E94B6350E94433D18
:1084F0001F910F91FF90EF90DF9008950F931F93BE
:10850000DF93CF93CDB7DEB760970FB6F894DEBF99
:108510000FBECDBF83E061E00E94334981E061E09E
:108520000E94334986E161E00E94334985E161E0C0
:108530000E94334983E061E00E94724981E061E07A
:108540000E9472491092920B1092930B1092940B0E
:108550001092950B1092960B1092970B0E9416405A
:1085600081E060E00E94724980E061E00E9433494E
:1085700080E061E00E9472498AE598E060E00E9434
:10858000952011E0109381008CE061E00E94334956
:108590008DE061E00E943349609136028DE070E029
:1085A0000E94194A80913B026FEF70E0681B7109CD
:1085B0008CE00E94194A89E79BE060E142E020E0FC
:1085C0000E9444488BE060E00E9433498BE061E008
:1085D0000E9472498BEE9BE00E94964480918E0B24
:1085E0008160817880938E0B10928F0B1093900B8B
:1085F00088E08093910B10929E0B10929F0B10922B
:10860000A00B1092A10BDE011196E7E9F2E00190B8
:108610000D928150E1F7DE011996EFE8F2E088E073
:1086200001900D928150E1F789E79BE061E08E01B6
:108630000F5F1F4FA8010E94C9471A821B8281E069
:108640008C8389E79BE060E0A8010E94C94789E725
:108650009BE062E0AE01475F5F4F0E94C9478CE13B
:1086600061E00E9433498CE160E00E9472498FE131
:1086700060E00E9433498EE160E00E9433498DE161
:1086800060E00E9433498FE161E00E9472498EE10F
:1086900061E00E9472498DE161E00E9472490E948E
:1086A0002B3A882329F480918E0B806280938E0B65
:1086B00060960FB6F894DEBF0FBECDBFCF91DF91AD
:1086C0001F910F9108950F931F93DF93CF93CDB711
:1086D000DEB728970FB6F894DEBF0FBECDBFFC0102
:1086E0008B0180913102858384E893E0BF0144E0EF
:1086F0000E94972C882311F490E032C01093A601B9
:108700000093A5018091BE01882319F00E94F529EC
:1087100021C08091C30189838091C8018A8380919F
:10872000CD018B838091D2018C838091D7018D8381
:108730008091DC018E838091E1018F838091E6013D
:108740008887CE010196BE016B5F7F4F40E050E00D
:108750000E94742C90E0882309F491E081E098272E
:10876000892F28960FB6F894DEBF0FBECDBFCF91EC
:10877000DF911F910F91089581E08093EA0B609340
:10878000C70B1092E80B1092E90B08952091C60BCD
:1087900030E08091C50B281B3109C9010895409133
:1087A000C50B8091C60B481718F02FEF3FEF0AC09A
:1087B000E42FF0E0EB55F44F8081282F30E04F5F3D
:1087C0004093C50BC9010895E091C50B8091C60B7C
:1087D000E81718F0EFEFFFEF06C0F0E0EB55F44FAD
:1087E0008081E82FF0E0CF01089508951092EE0BFC
:1087F0001092ED0B88EE93E0A0E0B0E08093EF0BD9
:108800009093F00BA093F10BB093F20B83EA92E0FC
:108810009093EC0B8093EB0B0895CF92DF92EF9245
:10882000FF920F931F93CF93DF937C016B018A011B
:108830008091EA0B8823A1F0C0E0D0E00DC0D70101
:10884000ED91FC91D601AC0FBD1F0190F081E02DA0
:10885000C7016C9109952196C017D10780F304C018
:10886000CB01642F0E943F45C801DF91CF911F913A
:108870000F91FF90EF90DF90CF900895DF93CF930B
:108880000F92CDB7DEB7FC0169838091EA0B882394
:10889000C9F08091E90B803238F081E090E0938359
:1088A000828320E030E015C08091E80BE82FF0E0F3
:1088B000E853F44F998190838F5F8093E80B809306
:1088C000E90B05C0CE01019661E00E943F4521E021
:1088D00030E0C9010F90CF91DF9108950F93062FDB
:1088E0008091C70B68EC7BE04091E90B21E00E948E
:1088F000EA441092E80B1092E90B1092EA0B0F91E8
:10890000089561E00E946E440895413208F040E20B
:10891000862F65EA7BE00E94A1441092C50B8093EC
:10892000C60B089521E00E94854408951092C50B5E
:108930001092C60B1092E80B1092E90B0E94EB46C6
:108940000895382F413210F040E042C08091F70B7B
:108950008823E1F791E09093F70B2093F90B8FEFC9
:108960008093640C10921F0C41504093200C4F5F79
:108970009093F80B8091F80B330F832B8093F80BB7
:108980008091FA0B813041F41092FA0B8091F80B30
:108990008093BB0085EC01C085EE8093BC00809184
:1089A000F70B8130E1F380911F0C841710F4409194
:1089B0001F0C20E030E00AC0FB01E20FF31FD901D9
:1089C000A150B44F8C9180832F5F3F4F2417A0F3A9
:1089D000842F08950F931F93582F122F413210F0B8
:1089E00081E04AC08091F70B8823E1F782E0809311
:1089F000F70B0093F90B8FEF8093640C10921F0C10
:108A00004093200CAFEFBBE0FB0102C081918D933E
:108A10008E2F861B8417D0F31092F80B8091F80BE1
:108A2000550F852B8093F80B8091FA0B813041F420
:108A30001092FA0B8091F80B8093BB0085EC01C07B
:108A400085EE8093BC00112321F08091F70B8230DA
:108A5000E1F38091640C8F3F11F480E00DC08091B0
:108A6000640C803211F482E007C08091640C803382
:108A700011F084E001C083E01F910F910895482F09
:108A8000613210F081E008958091F70B843011F08D
:108A900082E008956093420CA1E2BCE0842F9C0127
:108AA000F90102C081918D938E2F841B8617D0F31C
:108AB00080E008951F920F920FB60F9211242F930A
:108AC0003F934F935F936F937F938F939F93AF9356
:108AD000BF93EF93FF938091B90090E0887F9070EF
:108AE0008036910509F4F2C081369105CCF58832C3
:108AF000910509F47BC089329105B4F48031910568
:108B000009F46FC0813191053CF4009709F447C125
:108B1000089709F04FC165C08831910509F466C016
:108B2000809709F047C182C08034910509F4A4C040
:108B30008134910544F48033910509F482C0C897CB
:108B400009F038C189C08035910509F489C088359C
:108B5000910509F496C08834910509F02BC1AEC087
:108B60008839910509F413C189399105ECF48837E6
:108B7000910509F4ABC0893791054CF4883691050D
:108B800009F4A4C08037910509F014C19FC088384A
:108B9000910509F4FCC08039910509F49DC0803825
:108BA000910509F007C198C0803B910509F4C6C042
:108BB000813B91054CF4803A910509F49FC0883AB5
:108BC000910509F0F7C0BAC0803C910509F4E3C0F3
:108BD000883C910509F4DFC0883B910509F0EAC0A3
:108BE000C2C08091F80B8093BB00CFC090911F0C46
:108BF0008091200C981768F490911F0CE92FF0E0F9
:108C0000E150F44F80818093BB009F5F90931F0CD5
:108C1000BCC08091F90B882309F44BC085ED80938B
:108C2000BC008091BC0084FDFCCFC2C080E2809378
:108C3000640C85ED8093BC008091BC0084FDFCCF6A
:108C4000B7C080E38093640C85ED8093BC00809175
:108C5000BC0084FDFCCFACC088E38093640C9BC057
:108C600080911F0C9091BB00E82FF0E0E150F44F91
:108C700090838F5F80931F0C90911F0C8091200C2C
:108C800082C080911F0C9091BB00E82FF0E0E15072
:108C9000F44F90838F5F80931F0C8091F90B882392
:108CA00041F085ED8093BC008091BC0084FDFCCF39
:108CB0007FC081E08093FA0B84EA6EC085ED8093DB
:108CC000BC008091BC0084FDFCCF72C083E0809327
:108CD000F70B1092630C59C08091630C803208F03E
:108CE00056C08091630C9091BB00E82FF0E0ED5BE3
:108CF000F34F90838F5F8093630C47C08091630C28
:108D0000803230F4E091630CF0E0ED5BF34F1082C1
:108D100085ED8093BC008091BC0084FDFCCF109257
:108D2000F70B6091630CE091FD0BF091FE0B83E477
:108D30009CE070E009951092630C2DC084E0809354
:108D4000F70B1092410C1092420CE091FB0BF0914A
:108D5000FC0B09958091420C882329F481E08093D3
:108D6000420C1092210C9091410CE92FF0E0EF5D44
:108D7000F34F80818093BB009F5F9093410C909153
:108D8000410C8091420C981710F485EC01C085E8E5
:108D90008093BC000FC085EC8093BC0009C010928A
:108DA000640C85ED8093BC008091BC0084FDFCCFF9
:108DB0001092F70BFF91EF91BF91AF919F918F911F
:108DC0007F916F915F914F913F912F910F900FBEC7
:108DD0000F901F9018951092F70B81E08093F90B7C
:108DE0001092FA0B81E161E00E94724980E161E03A
:108DF0000E947249E9EBF0E080818E7F8083808160
:108E00008D7F808380E28093B80085E48093BC00EE
:108E100008950F931F938C01FC01868160E00E94EE
:108E2000724981E090E00E94344BF801868161E054
:108E30000E94724981E090E00E94344BF8018681E3
:108E400060E00E94724984E690E00E94344B1F91DA
:108E50000F910895CF92DF92EF92FF920F931F939D
:108E6000CF93DF93D82EC92E282F392FC9018C011B
:108E7000C0E0D0E0E62EFF24F801878161E00E9487
:108E80003349B7010C2E02C0759567950A94E2F735
:108E90006170F80187810E94724921960F5F1F4F10
:108EA000C830D10549F78D2D9C2D0E940947DF91CF
:108EB000CF911F910F91FF90EF90DF90CF90089589
:108EC000CF92DF92EF92FF920F931F93CF93DF9396
:108ED000D82EC92E282F392FC9018C01C0E0D0E02F
:108EE000E62EFF24F801878161E00E943349B70133
:108EF0000C2E02C0759567950A94E2F76170F8012F
:108F000087810E94724921960F5F1F4FC430D1059F
:108F100049F78D2D9C2D0E940947DF91CF911F911C
:108F20000F91FF90EF90DF90CF9008951F93CF9314
:108F3000DF93EC01162F8C81642F0E9472498D8182
:108F40008F3F19F060E00E9472498F8584FF05C051
:108F5000CE01612F0E942A470EC0612F70E084E08D
:108F6000759567958A95E1F7CE010E946047CE011D
:108F7000612F0E946047DF91CF911F91089541E0DA
:108F80000E94964781E090E0089540E00E94964755
:108F90000895EF92FF920F931F93CF93DF938C016D
:108FA0007A016770660F660F660F60640E94C5479E
:108FB000C0E0D0E0D801ED91FC91D701AC0FBD1F0E
:108FC0000190F081E02DC8016C9109952196C8307F
:108FD000D10581F7DF91CF911F910F91FF90EF9015
:108FE0000895FC016089862F8160808B6960CF01C4
:108FF0000E94C5470895FC0160896E7F608B6860A0
:109000000E94C5470895FC016089862F8460808B8B
:109010006C60CF010E94C5470895DF93CF93CDB711
:10902000DEB728970FB6F894DEBF0FBECDBF9C0108
:10903000FE013196A7EBB2E088E00D9001928150DD
:10904000E1F7F9018389481710F0482F4150E42FC8
:10905000F0E0EE0FFF1FEC0FFD1F8181680F6068CD
:10906000C9010E94C54728960FB6F894DEBF0FBE0F
:10907000CDBFCF91DF91089561E00E94C54780ED9B
:1090800097E00E94344B0895CF93DF93EC01423078
:1090900018F08F8588608F874B8B1C8A222329F0DC
:1090A000413019F48F8584608F8780E593EC0E94AE
:1090B000344B8C8160E00E9472498E8160E00E9496
:1090C00072498D818F3F19F060E00E9472496F856F
:1090D00064FD1DC0CE0163E00E94604784E991E118
:1090E0000E94344BCE0163E00E94604784E991E125
:1090F0000E94344BCE0163E00E94604786E990E015
:109100000E94344BCE0162E00E94604716C060624C
:10911000CE010E94C54784E991E10E94344B6F85DE
:109120006062CE010E94C54786E990E00E94344B00
:109130006F856062CE010E94C5476F856062CE0177
:109140000E94C54784E0888BCE010E940348CE016F
:109150000E943C4882E0898BCE0166E00E94C547B0
:10916000DF91CF9108956F927F928F92AF92CF92BD
:10917000EF920F931F93DF93CF93CDB7DEB73C01F0
:10918000162F842FF301448325830683E782C0864C
:10919000A18682869D8593879E8594879F859587E6
:1091A0009889968761E00E943349F30185818F3F5A
:1091B00019F061E00E943349F301868161E00E9469
:1091C0003349112319F0F301178603C080E1F3013D
:1091D0008787C30160E141E020E00E944448CF91CD
:1091E000DF911F910F91EF90CF90AF908F907F9074
:1091F0006F9008958F92AF92CF92EF920F931F933B
:10920000CF93DF93DC01362F542F722F102FAE2C0B
:109210008C2C13961C921E92129783EB92E011965F
:109220009C938E9300D000D0EDB7FEB73196CDB7AA
:10923000DEB71982118212821382CD0161E0432FC1
:109240002FEF052FE72EC12E0E94B3480F900F90ED
:109250000F900F90DF91CF911F910F91EF90CF90D2
:10926000AF908F900895CF93DF93482F50E0CA01BD
:109270008C53944FFC0134914C55544FFA01849116
:10928000882369F190E0880F991FFC01EA57F44F99
:10929000A591B491FC01E057F44FC591D491662398
:1092A00051F42FB7F8948C91932F909589238C9338
:1092B000888189230BC0623061F42FB7F8948C91B8
:1092C000932F909589238C938881832B88832FBF3C
:1092D00006C09FB7F8948C91832B8C939FBFDF912E
:1092E000CF910895482F50E0CA018C51944FFC0152
:1092F0002491CA018C53944FFC0194914C55544FC6
:10930000FA013491332309F440C0222351F1233070
:1093100071F0243028F42130A1F0223011F514C06E
:109320002630B1F02730C1F02430D9F404C0809148
:1093300080008F7703C0809180008F7D80938000B4
:1093400010C084B58F7702C084B58F7D84BD09C0FD
:109350008091B0008F7703C08091B0008F7D8093A3
:10936000B000E32FF0E0EE0FFF1FE057F44FA591A0
:10937000B4912FB7F894662321F48C9190958923AA
:1093800002C08C91892B8C932FBF0895682F70E0B9
:10939000CB018C51944FFC012491CB018C53944F01
:1093A000FC0144916C55744FFB019491992319F47D
:1093B00020E030E03CC0222351F1233071F0243012
:1093C00028F42130A1F0223011F514C02630B1F07C
:1093D0002730C1F02430D9F404C0809180008F7709
:1093E00003C0809180008F7D8093800010C084B581
:1093F0008F7702C084B58F7D84BD09C08091B00095
:109400008F7703C08091B0008F7D8093B000892F4B
:1094100090E0880F991F8656944FFC01A591B49156
:109420008C9120E030E0842311F021E030E0C9018C
:1094300008951F93CF93DF93182FEB0161E00E94F3
:109440003349209709F44AC0CF3FD10509F449C0F8
:10945000E12FF0E0EC51F44F84918330C1F084307F
:1094600028F4813051F08230B1F50CC0863019F10A
:10947000873049F1843079F514C084B5806884BDA3
:10948000C7BD33C084B5806284BDC8BD2EC0809185
:109490008000806880938000D0938900C09388000A
:1094A00024C080918000806280938000D0938B00E4
:1094B000C0938A001AC08091B00080688093B00089
:1094C000C093B30012C08091B00080628093B0005E
:1094D000C093B4000AC0C038D1051CF4812F60E0ED
:1094E00002C0812F61E00E947249DF91CF911F91EC
:1094F00008951F920F920FB60F9211242F933F934E
:109500004F935F936F937F938F939F93AF93BF938B
:109510002091690C30916A0C40916B0C50916C0C4D
:1095200070916D0CDA01C9010296A11DB11D672F62
:109530006A5F6D3730F06D57DA01C9010396A11DDE
:10954000B11D60936D0C8093690C90936A0CA0938D
:109550006B0CB0936C0C8091650C9091660CA09193
:10956000670CB091680C0196A11DB11D8093650C2C
:109570009093660CA093670CB093680CBF91AF9169
:109580009F918F917F916F915F914F913F912F911B
:109590000F900FBE0F901F9018958FB7F8942091E1
:1095A000690C30916A0C40916B0C50916C0C8FBF20
:1095B000B901CA0108959B01AC017FB7F89480916D
:1095C000650C9091660CA091670CB091680C66B523
:1095D000A89B05C06F3F19F00196A11DB11D7FBF6B
:1095E000BA2FA92F982F8827860F911DA11DB11D75
:1095F00063E0880F991FAA1FBB1F6A95D1F7BC01B2
:109600002DC0FFB7F8948091650C9091660CA091E5
:10961000670CB091680CE6B5A89B05C0EF3F19F048
:109620000196A11DB11DFFBFBA2FA92F982F882722
:109630008E0F911DA11DB11DE3E0880F991FAA1F78
:10964000BB1FEA95D1F7861B970B885E9340C8F243
:10965000215030404040504068517C4F2115310529
:109660004105510571F60895019739F0019729F0E8
:10967000880F991F01970197F1F70895789484B5A1
:10968000826084BD84B5816084BD85B5826085BDFE
:1096900085B5816085BDEEE6F0E0808181608083E4
:1096A000E1E8F0E0108280818260808380818160C7
:1096B0008083E0E8F0E0808181608083E1EBF0E08E
:1096C000808184608083E0EBF0E080818160808332
:1096D000EAE7F0E08081846080838081826080831B
:1096E0008081816080838081806880831092C10046
:1096F0000895CF93DF930E943E4B0E94CE1CCAEB8D
:10970000DCE40E947D1D2097E1F30E94BA4CF9CF62
:10971000CF92DF92EF92FF920F931F93CF93DF933D
:109720007C016B018A01C0E0D0E00FC0D6016D91D1
:109730006D01D701ED91FC910190F081E02DC70101
:109740000995C80FD91F015010400115110571F777
:10975000CE01DF91CF911F910F91FF90EF90DF909D
:10976000CF900895DC01ED91FC910190F081E02D06
:1097700009950895CF93DF93DB010D900020E9F761
:109780001197A61BB70BEC01E881F9810280F381E8
:10979000E02DAD010995DF91CF9108954F925F9231
:1097A0007F928F929F92AF92BF92CF92DF92EF9271
:1097B000FF920F931F93DF93CF93CDB7DEB7A1979F
:1097C0000FB6F894DEBF0FBECDBF2C01742ECB01B7
:1097D000223008F42AE019A231E2C32ED12CCC0E9B
:1097E000DD1E822E9924AA24BB24672D752FA50186
:1097F00094010E94404F79018A01C801B701A50177
:1098000094010E94EE4E472D461B0894C108D108D2
:109810004A3014F4405D01C0495CF6014083E11414
:10982000F1040105110521F07E2C5F2DC801DDCF6B
:10983000C201B6010E94BA4BA1960FB6F894DEBFE2
:109840000FBECDBFCF91DF911F910F91FF90EF9091
:10985000DF90CF90BF90AF909F908F907F905F9060
:109860004F900895CF92DF92EF92FF920F931F9344
:10987000CF93DF93EC016A017B012115310541F49F
:10988000E881F9810190F081E02D642F09951FC0D6
:109890002A303105D1F477FF17C0E881F9810190B2
:1098A000F081E02D6DE209958C0144275527BA011E
:1098B0004C195D096E097F09CE012AE00E94CE4B4A
:1098C0009801280F391F04C02AE00E94CE4B9C014A
:1098D000C901DF91CF911F910F91FF90EF90DF9021
:1098E000CF900895EF92FF920F931F937B019A01FF
:1098F0000027F7FC0095102FB801A7010E94324CF9
:109900001F910F91FF90EF90089508951F920F926D
:109910000FB60F9211242F933F934F938F939F93E2
:10992000EF93FF934091C6002091AE0C3091AF0CA5
:109930002F5F3F4F2F7330708091B00C9091B10C1E
:109940002817390759F0E091AE0CF091AF0CE259AD
:10995000F34F40833093AF0C2093AE0CFF91EF9107
:109960009F918F914F913F912F910F900FBE0F902C
:109970001F901895E091020DF091030DE05CFF4FF0
:109980008191919120813181821B930B8F73907013
:10999000892B11F00E94854C08951F920F920FB6EB
:1099A0000F9211242F933F938F939F93EF93FF93E5
:1099B0002091F20C3091F30C8091F40C9091F50C05
:1099C0002817390731F48091C1008F7D8093C10041
:1099D00014C0E091F40CF091F50CEE54F34F20819B
:1099E0008091F40C9091F50C01968F739070909388
:1099F000F50C8093F40C2093C600FF91EF919F919A
:109A00008F913F912F910F900FBE0F901F9018953F
:109A1000DC011C96ED91FC911D97E05CFF4F2191BC
:109A2000319180819181281B390B2F733070C901CE
:109A30000895DC011C96ED91FC911D97E05CFF4FB1
:109A400020813181E054F040DF01AE5BBF4F8D914A
:109A50009C9111972817390719F42FEF3FEF07C092
:109A60008D919C91E80FF91F8081282F30E0C9016A
:109A70000895DC011C96ED91FC911D97E05CFF4F71
:109A800020813181E054F040DF01AE5BBF4F8D910A
:109A90009C9111972817390719F42FEF3FEF10C049
:109AA0008D919C911197E80FF91F20818D919C91C8
:109AB000119701968F73907011969C938E9330E05E
:109AC000C9010895FC0186859785DC01A05CBF4F24
:109AD000FC01EE5BFF4F2D913C91119780819181AC
:109AE00028173907C1F70895CF93DF93EC01EE856E
:109AF000FF85E05CFF4F20813181E054F0402F5F13
:109B00003F4F2F733070DF01AE5BBF4F8D919C9143
:109B1000119728173907D1F3E05CFF4F80819181BD
:109B2000E054F040E80FF91F6083EE85FF85E05CAC
:109B3000FF4F31832083EE89FF89208181E090E00F
:109B40000D8C02C0880F991F0A94E2F7282B2083FE
:109B500081E090E0DF91CF9108951092F90C10927E
:109B6000F80C88EE93E0A0E0B0E08093FA0C9093BC
:109B7000FB0CA093FC0CB093FD0C83EC92E0909353
:109B8000F70C8093F60C8EE69CE09093030D809387
:109B9000020D82EB9CE09093050D8093040D85EC03
:109BA00090E09093070D8093060D84EC90E09093E5
:109BB000090D8093080D80EC90E090930B0D80933D
:109BC0000A0D81EC90E090930D0D80930C0D86ECC6
:109BD00090E090930F0D80930E0D84E08093100D14
:109BE00083E08093110D87E08093120D85E08093D0
:109BF000130D81E08093140D0895E89409C097FB3C
:109C00003EF490958095709561957F4F8F4F9F4F53
:109C10009923A9F0F92F96E9BB279395F695879597
:109C200077956795B795F111F8CFFAF4BB0F11F45A
:109C300060FF1BC06F5F7F4F8F4F9F4F16C0882301
:109C400011F096E911C0772321F09EE8872F762F37
:109C500005C0662371F096E8862F70E060E02AF078
:109C60009A95660F771F881FDAF7880F9695879564
:109C700097F9089597F99F6780E870E060E008958C
:109C80009FEF80EC089500240A9416161706180614
:109C90000906089500240A941216130614060506F0
:109CA0000895092E0394000C11F4882352F0BB0F81
:109CB00040F4BF2B11F460FF04C06F5F7F4F8F4FE4
:109CC0009F4F089557FD9058440F551F59F05F3F1F
:109CD00071F04795880F97FB991F61F09F3F79F0CE
:109CE00087950895121613061406551FF2CF469550
:109CF000F1DF08C0161617061806991FF1CF8695D2
:109D00007105610508940895E894BB2766277727B5
:109D1000CB0197F908950BD0C4CFB5DF28F0BADF97
:109D200018F0952309F0A6CFABCF1124EECFCADFF0
:109D3000A0F3959FD1F3950F50E0551F629FF0015E
:109D4000729FBB27F00DB11D639FAA27F00DB11DB7
:109D5000AA1F649F6627B00DA11D661F829F222740
:109D6000B00DA11D621F739FB00DA11D621F839FC7
:109D7000A00D611D221F749F3327A00D611D231F9D
:109D8000849F600D211D822F762F6A2F11249F57EB
:109D900050408AF0E1F088234AF0EE0FFF1FBB1F0E
:109DA000661F771F881F91505040A9F79E3F5105AD
:109DB00070F060CFAACF5F3FECF3983EDCF386955E
:109DC00077956795B795F795E7959F5FC1F7FE2B58
:109DD000880F911D9695879597F90895629FD001F8
:109DE000739FF001829FE00DF11D649FE00DF11D56
:109DF000929FF00D839FF00D749FF00D659FF00D05
:109E00009927729FB00DE11DF91F639FB00DE11DF1
:109E1000F91FBD01CF0111240895991B79E004C0F9
:109E2000991F961708F0961B881F7A95C9F7809599
:109E30000895AA1BBB1B51E107C0AA1FBB1FA61791
:109E4000B70710F0A61BB70B881F991F5A95A9F7E3
:109E500080959095BC01CD01089597FB092E0726AA
:109E60000AD077FD04D0E5DF06D000201AF4709503
:109E700061957F4F0895F6F7909581959F4F0895CE
:109E8000A1E21A2EAA1BBB1BFD010DC0AA1FBB1FFE
:109E9000EE1FFF1FA217B307E407F50720F0A21B70
:109EA000B30BE40BF50B661F771F881F991F1A94DD
:109EB00069F760957095809590959B01AC01BD0107
:109EC000CF010895EE0FFF1F0590F491E02D099446
:109ED0002F923F924F925F926F927F928F929F92BA
:109EE000AF92BF92CF92DF92EF92FF920F931F93A8
:109EF000CF93DF93CDB7DEB7CA1BDB0B0FB6F89459
:109F0000DEBF0FBECDBF09942A88398848885F8498
:109F10006E847D848C849B84AA84B984C884DF8009
:109F2000EE80FD800C811B81AA81B981CE0FD11DED
:109F30000FB6F894DEBF0FBECDBFED010895F894C3
:029F4000FFCF51
:109F420074007077006C6F63006E707700637077D7
:109F5200007069640064006D007900763D5B0072F8
:109F6200736E0072627400656E006D6D0072640043
:109F7200743D5B006F70656E646F6F7200426F7349
:109F8200746F6E2C4D41000069692D30007B4901D0
:109F9200531A4C0180174F018D1352016E1855014F
:109FA200051958011A165B011D0A5E01C7106101ED
:109FB200410E6401CF1767010A106A011C126D017C
:109FC2009C0870014C1B7301E60F41726475696E47
:109FD2006F2D3030003703010306FF638253633570
:109FE200010405060750000100010A100E0000C915
:109FF200004A0900206C58090301016309010101AB
:10A002006D0901C0FF770901A8FF83090101FF88DB
:10A01200090116FF8D0901C0FF920901A8FF9F09DE
:10A022000101FFA4090101FFA9090150FFAE0902C4
:10A0320000FFB909020101BA09010005CA090301B9
:10A0420001D7090300F0E309030008F20903003C09
:10A05200020A033C78100A0300011F0A03010130BF
:10A062000A0364FA3F0A030AF04D0A0100015C0A7E
:10A072000300FF6D0A016EFF780A01C8FF860A011C
:10A08200CCFF950A0109FFA50A0136FFAA0A01774A
:10A09200FFAF0A010001B40A01BF0AC30AC70ACB13
:10A0A2000ACF0AD30AD70A000000003607884B6F8E
:10A0B200000000002E6F4FFFFFFFFFFFFFFFFFFFBB
:10A0C200FFFFFF1F1C1F1E1F1E1F1F1E1F1E1F0024
:10A0D200001F111F11131E0014081501050515009C
:10A0E2000000003E440D44C643CF43E443F5430021
:10A0F200000000BF47884B000040001400540000DD
:10A10200000000744D884B084D394D194D624D00C9
:00000001FF
